:100000000C94EF020C940C030C940C030C940C0352
:100010000C940C030C940C030C940C030C940C0324
:100020000C940C030C9453110C940C030C94341189
:100030000C94091E0C940C030C940C030C940C03EC
:100040000C940C030C940C030C94B40F0C940C0340
:100050000C94C20B0C940C030C943F060C940C03F0
:100060000C9459120C940C030C943E1D0C940C032C
:100070005B1D621D761D831D901D881D901DA21D98
:10008000CC1DB31DB71DD71DC11DCC1DBA1DBE1D76
:10009000D71DC11DCC1DD01DD41DD71DDB1D0A0AC7
:1000A0000D004E65757472616C0048656164696E1F
:1000B00067486F6C64000A0D537465756572756EE0
:1000C000673A20004F4B0A0D000A0D4162676C65CC
:1000D000696368204C756674647275636B73656ED2
:1000E000736F722E2E000A0D42656E75747A65204C
:1000F000506172616D657465727361747A202564F4
:10010000000A0D414343206E696368742061626791
:1001100065676C696368656E21000A0D496E6974D4
:100120002E20454550524F4D3A2047656E6572610D
:1001300074696E672044656661756C742D506172D8
:10014000616D65746572207573696E67206F6C648C
:1001500020537469636B2053657474696E67730010
:100160000A0D496E69742E20454550524F4D3A2074
:1001700047656E65726174696E6720446566617576
:100180006C742D506172616D6574657220616E646E
:1001900020537469636B2D53657474696E67732E95
:1001A0002E2E000A0D3D3D3D3D3D3D3D3D3D3D3D3D
:1001B0003D3D3D3D3D3D3D3D3D3D3D3D3D3D3D3D6F
:1001C0003D3D3D000A0D466C69676874436F6E746F
:1001D000726F6C0A0D48617264776172653A2564CA
:1001E0002E25640A0D536F6674776172653A562541
:1001F000642E2564256320002E0048693A25346961
:10020000202043663A253469200047733A25346933
:10021000202047693A25346920004E693A2534691F
:100220002020526F3A253469200045787465726E3B
:10023000436F6E74726F6C20200052616E67653A76
:100240002533692D253369005374656C6C756E67B1
:100250003A2025336900536574706F696E742020ED
:1002600025336900536572766F202000506F7469E2
:10027000343A202025336900506F7469333A2020C6
:1002800025336900506F7469323A202025336900A4
:10029000506F7469313A20202533690053746172BC
:1002A000743A2020202020253569004D657373772E
:1002B0006572743A20202535690052696368747547
:1002C0006E673A2020253569004B6F6D706173733E
:1002D0002020202020202000456D70662E5065676C
:1002E000656C3A253569005370616E6E756E673ABC
:1002F000202025356900486F63682025346920284F
:100300002533692900526F6C6C202534692028251B
:10031000336929004E69636B202534692028253311
:10032000692900414343202D2053656E736F72008D
:1003300047696572202534692028253369292825D5
:1003400033692900526F6C6C2025346920282533CD
:1003500069292825336929004E69636B2025346992
:1003600020282533692928253369290047696572C2
:100370002025346920282533692900526F6C6C20B0
:10038000253469202825336929004E69636B2025AF
:10039000346920282533692900476965722025348E
:1003A0006920282533692900526F6C6C2025346937
:1003B000202825336929004E69636B202534692084
:1003C0002825336929004779726F202D2053656EE7
:1003D000736F720050333A253469202050343A2527
:1003E0003469200050313A253469202050323A25B2
:1003F0003469200047733A253469202047693A253B
:10040000346920004E693A2534692020526F3A251C
:10041000346920004B373A25346920204B383A257F
:10042000346920004B353A25346920204B363A2573
:10043000346920004B333A25346920204B343A2567
:10044000346920004B313A25346920204B323A255B
:10045000346920004B6F6D706173733A2020202542
:10046000356900526F6C6C3A202020202020253501
:1004700069004E69636B3A202020202020253569D1
:1004800000616B742E204C6167650048F668656EEC
:10049000726567656C756E67004B65696E652000F7
:1004A0004F66662020202020203A20253569004C08
:1004B000756674647275636B3A2025356900536FF5
:1004C0006C6C486F6568653A2025356900486F6532
:1004D00068653A20202020202535690028632920DE
:1004E000486F6C676572204275737300536574744E
:1004F000696E673A202564200048573A5625642ED5
:1005000025642053573A25642E25642563002B204B
:100510004D696B726F4B6F70746572202B005B2599
:10052000695D005B25695D00000011002300340057
:100530004600570069007A008B009C00AE00BF00A7
:10054000D000E100F200030114012401350146014D
:1005500056016601770187019701A701B601C6011F
:10056000D501E501F4010302120221022F023E022D
:100570004C025A0268027502830290029D02AA028E
:10058000B702C302CF02DB02E702F302FE02090355
:1005900014031F03290333033D0347035003590387
:1005A00062036B0373037B0383038A039203990340
:1005B0009F03A603AC03B203B703BC03C103C60386
:1005C000CA03CE03D203D603D903DC03DE03E1035F
:1005D000E303E403E603E703E703E803E803112486
:1005E0001FBECFEFD0E1DEBFCDBF13E0A0E0B1E092
:1005F000E0E3F0EB02C005900D92A83BB107D9F7FC
:1006000019E0A8EBB3E001C01D92A836B107E1F7ED
:100610000E94D4030C9416580C9400009C01F99984
:10062000FECF32BD21BDF89A80B508959C01F9999D
:10063000FECF1FBA32BD21BD60BD0FB6F894FA9A45
:10064000F99A0FBE0895F999FECF22E030E032BD4D
:1006500021BDF89A90B5892F8150853068F0F999BD
:10066000FECF1FBA32BD21BD83E080BD0FB6F89426
:10067000FA9AF99A0FBE93E0892F0895282F8630B1
:1006800010F025E002C0882369F0F999FECF1FBA67
:1006900082E090E092BD81BD20BD0FB6F894FA9A39
:1006A000F99A0FBE08958091B007A82FB0E0FD0120
:1006B000EE0FFF1FE258F84F808191818D5E9F4FB2
:1006C00014F010920201AA0FBB1FA258B84F8D91CF
:1006D0009C918A5B9F4FBCF480910201882399F41E
:1006E00081E08093020180917B068F5F80937B067F
:1006F000853038F088EE93E09093DA038093D90345
:1007000002C00E94D52880917B06809348071092F2
:10071000490708951F93182F863010F015E002C086
:10072000882319F1812F90E00197242F30E0FC01FC
:10073000E29FC001E39F900DF29F900D112426E1EE
:1007400033E050E08C599F4F0E941955F999FECF24
:100750001FBA82E090E092BD81BD10BD0FB6F89443
:10076000FA9AF99A0FBE0E9470541F910895982F1B
:10077000FB018150853008F093E0892F90E00197CC
:10078000242F30E0829FB001839F700D929F700DE7
:1007900011246C597F4F2EE033E050E0CF010E94CE
:1007A000FD540E94705408957F928F929F92AF9251
:1007B000BF92CF92DF92EF92FF920F931F93CF934E
:1007C000DF9314B815B8189B08C0199B02C08DE0C0
:1007D00001C08BE08093000109C0199B02C084E135
:1007E000F9CF8AE0809300018DEC87B93E9A8FEFB4
:1007F00088B98BE184B981E085B98EE38AB9579ACB
:1008000087E78BB984B7877F84BF80916000886158
:10081000809360001092600080ED97E09093DA037F
:100820008093D9031092830410928204109283075C
:1008300010928207109281041092800410927F041B
:1008400010927E04809100018A3011F0843111F4FD
:10085000289801C0289A0E94C7100E9411070E9480
:10086000F41D0E9453120E94001D0E94875178942B
:100870002091000188E690E09F938F9387E490E0B9
:100880009F938F931F921F92822F6AE00E946F574F
:10089000892F90E09F938F93822F0E946F5790E053
:1008A0009F938F9384EC91E09F938F931F920E946C
:1008B000F90C83EA91E09F938F931F920E94F90CA9
:1008C0008DB79EB740960FB6F8949EBF0FBE8DBFF2
:1008D000809100018C3010F4299A01C0299849E0D8
:1008E00060EB77E083E00E94B703F999FECFC1E0A7
:1008F000D0E0D2BDC1BDF89A80B58F3FC1F0F99963
:10090000FECFD2BDC1BDF89A80B5893480F0809108
:10091000B0078A3060F48091B1078A3040F480914A
:10092000B2078A3020F48091B3078A3050F080E615
:1009300091E09F938F931F920E94F90C0E94E51EF5
:100940000FC0F999FECFD2BDC1BDF89A80B58934E8
:1009500051F08AE191E09F938F931F920E94F90CCE
:100960000F900F900F90F999FECFD2BDC1BDF89AAC
:1009700080B5893409F431C00E94DF4611E012309D
:1009800039F0133019F40E949A4504C0143010F065
:100990000E943B4646E560EB77E0812F0E948A0388
:1009A0001F5F163061F7F999FECF1FBA82E090E021
:1009B00092BD81BD83E080BD0FB6F894FA9AF99A92
:1009C0000FBEF999FECF1FBAD2BDC1BD89E480BD6B
:1009D0000FB6F894FA9AF99A0FBEF999FECF84E00F
:1009E00090E092BD81BDF89A80B5853050F081E0ED
:1009F00091E09F938F931F920E94F90C0F900F909C
:100A00000F900E94230346E560EB77E00E94B70356
:100A10000E94230390E09F938F9386EE90E09F9334
:100A20008F931F920E94F90C8091B8070F900F903E
:100A30000F900F900F9080FD03C0C8EED3E020C050
:100A400089EC90E09F938F931F920E94F90C88EE9F
:100A500093E00E94EF10EC010E9409160F900F9096
:100A60000F90CE010E94F9108823D9F384EC90E016
:100A70009F938F931F920E94F90C0F900F900F90ED
:100A80000E94942A809100018A3011F0843111F47F
:100A9000289801C0289A80ED97E09093DA0380931C
:100AA000D90385E580937D0686EB90E09F938F9335
:100AB0001F920E94F90C8091B8070F900F900F9031
:100AC00082FF03C08AEA90E002C082EA90E09F932E
:100AD0008F931F920E94F90C0F900F900F908EE948
:100AE00090E09F938F931F920E94F90C0E946416CE
:100AF00088E893E1909392038093910381E080933F
:100B00007C060F900F900F9064E0762E50E7852EB4
:100B100057E1952EA12C43E0B42E35E0C32ED12C05
:100B200020E1E22E27E2F22E00E810E08091D603C9
:100B3000882309F49CC01092D60380917B068823F9
:100B400019F00E94530302C00E945D2C0E94EF28FE
:100B5000809100018A3011F0843111F4289801C08D
:100B6000289A80910501882321F081508093050106
:100B70000EC0109287061092A00410929F0410924B
:100B8000A2041092A1041092A4041092A3048091D4
:100B90007D04882329F080917D04815080937D0419
:100BA0008091910390919203892BD1F4D09292037A
:100BB000C09291030E940F1D80910B0390910C0332
:100BC0008F5F9F4FF9F4809186048823D9F0F092CB
:100BD000DA03E092D90310930C0300930B0312C0C5
:100BE0008091910390919203019790939203809347
:100BF0009103809100018A3011F0843111F428981A
:100C000001C0289A8091D603882321F08091860420
:100C1000882311F40E9402080E94CA09CE010E9492
:100C2000F910882311F12091110330911203809162
:100C3000C80790E0281739077CF480910B03909146
:100C40000C038F5F9F4F41F49092DA038092D90397
:100C5000B0920C03A0920B030E94AE537092DB0380
:100C600084E190E00E94EF10EC010E947F5480919B
:100C7000DB03882309F05ACF0E94EF5357CF1F920E
:100C80000F920FB60F9211248F939F93EF93FF93C0
:100C9000809103018823E1F48091D2039091D303E2
:100CA00001969093D3038093D203FC01E35CFA4F47
:100CB000E081ED3019F08639910539F41092D303B3
:100CC0001092D20381E080930301E093C60004C038
:100CD0001092D3031092D203FF91EF919F918F91C5
:100CE0000F900FBE0F901F901895DC0120E030E0B0
:100CF00040E050E008C0FA01E35CFA4F8081280F21
:100D0000311D4F5F5F4F4A175B07A8F33F70C90162
:100D100036E0969587953A95E1F7835CFD01E35CB3
:100D2000FA4F808311962F73235CFD01E35CFA4F29
:100D30002083A25CBA4F8DE08C93109203018091C6
:100D40003D058093C60008955091C303565033E08B
:100D500043E048C0E32FF0E0E657F94F80813F5F62
:100D6000E32FF0E0E657F94F20812D533F5FE32F4B
:100D7000F0E0E657F94F70813F5FE32FF0E033502A
:100D8000E657F94F6081922F92959F708D53880F8F
:100D9000880F892BE42FF0E0E657F94F8083E42F8A
:100DA000EF5F513081F0972F9D53F0E02295207F27
:100DB000892F86958695282BE657F94F2083E42FB7
:100DC000EE5F523011F44E2F10C03C5F5350F0E0F4
:100DD0009295990F990F907C6D53962BE657F94F8A
:100DE00090834D5F552309F0B5CF8DE896E0909341
:100DF000C5038093C40343504093C60308951F93D3
:100E0000182F8A3019F48DE00E94FF068091C000EF
:100E100085FFFCCF1093C60080E090E01F910895FD
:100E20000895E1ECF0E088E18083A0ECB0E08C91E3
:100E300082608C93808180688083808180648083DD
:100E40008AE28093C40080910701909108010E947A
:100E5000EF1090936A06809369068CED90E00E94F3
:100E6000EF10909389068093880610926B0687E4B2
:100E700080936C0687E080936F068AE080936D060E
:100E800010926E061092C5031092C4031092C6030E
:100E90000895DF92EF92FF920F931F93DF93CF930A
:100EA000CDB7DEB78B857C8593E290933D058F5956
:100EB00080933E058A8580933F05DE011D9677234A
:100EC00029F4EE24FF2440E050E007C0ED84FE84C6
:100ED000DE0151964F855889715030E003E010E0F3
:100EE0007EC0F701E30FF11D90813F5F41505040FC
:100EF00091F4772309F483C0FD013296ED90FC90C4
:100F0000DF0112960190F081E02D7150309709F4C5
:100F100075C0AF0130E0F701E30FF11DD0803F5FF6
:100F20004150504099F4772311F460E023C0FD0153
:100F30003296ED90FC90DF01129640815181715004
:100F40004115510511F460E014C030E0F701E30FE2
:100F5000F11D60813F5F4150504061F4772351F0B3
:100F6000FD013296ED90FC90DF0112964081518197
:100F7000715030E0892F86958695835CF801E35C9B
:100F8000FA4F80832D2D22952F70892F90E083704A
:100F90009070F4E0880F991FFA95E1F7282B235CF5
:100FA000F801E25CFA4F20838D2D90E08F709070F5
:100FB000880F991F880F991F262F22952695269511
:100FC0002370282B235CF801E15CFA4F20836F73B8
:100FD000635CF801E05CFA4F60830C5F1F4F4115C2
:100FE000510509F07ECFC8010E947506CF91DF91AF
:100FF0001F910F91FF90EF90DF90089530E060E037
:10100000DD24B8CF80910301882309F4C2C1809107
:10101000BA038823C1F1809103018823A1F10E94C2
:101020006D1684E190E09F938F938091BE0324E13D
:10103000829FC00111248A5D9C4F9F938F9381E012
:1010400090E09F938F938EEB93E09F938F9382E03A
:101050008F9381E08F9388E48F930E94490780915A
:10106000BE038F5F8093BE032DB73EB7255F3F4F12
:101070000FB6F8943EBF0FBE2DBF843010F0109213
:10108000BE031092BA038091B903882371F1809155
:101090000301882351F10E946D1680E590E09F9333
:1010A0008F9386E293E09F938F9321E030E03F930C
:1010B0002F9386E793E09F938F933F932F938BE03B
:1010C00094E09F938F9383E08F9381E08F938CE4E0
:1010D0008F930E9449071092B9038DB79EB70F9660
:1010E0000FB6F8949EBF0FBE8DBF8091BC038823BE
:1010F000F1F0809103018823D1F08AE090E09F9382
:101100008F938BE696E09F938F9381E08F938F93DD
:1011100086E58F930E9449071092BC032DB73EB716
:10112000295F3F4F0FB6F8943EBF0FBE2DBF809191
:10113000B8038823F9F0809103018823D9F08BE06C
:1011400090E09F938F938DE796E09F938F9381E03C
:101150008F93809106018F9387E48F930E944907B4
:101160001092B8038DB79EB707960FB6F8949EBF3E
:101170000FBE8DBF80918806909189060E94F9105C
:10118000882309F459C080910301882309F454C0CD
:1011900060912A0470912B0480912C0490912D046D
:1011A0002CE630E040E050E00E94C45730937606D1
:1011B0002093750660913204709133048091340459
:1011C000909135042CE630E040E050E00E94C45796
:1011D0003093780620937706809195048093790662
:1011E0008091960480937A0688E090E09F938F9395
:1011F00085E796E09F938F9381E08F9383E08F93B1
:1012000087E78F930E9449072DB73EB7295F3F4F6D
:101210000FB6F8943EBF0FBE2DBF80917B06853080
:1012200018F086E080937B0683E690E00E94EF1042
:101230009093890680938806809107019091080118
:10124000892B41F08091690690916A060E94F910FD
:10125000882321F48091BB03882351F180910301FD
:10126000882331F182E490E09F938F9380E297E0AE
:101270009F938F9381E08F938F9384E48F930E9449
:1012800049071092BB0380910701909108012DB787
:101290003EB7295F3F4F0FB6F8943EBF0FBE2DBF3C
:1012A000009731F00E94EF1090936A0680936906D0
:1012B000209104012F3F51F180E190E09F938F93A3
:1012C000822F90E0A4E0880F991FAA95E1F7875F2D
:1012D0009E4F9F938F9381E090E09F938F9384E044
:1012E00091E09F938F9382E08F9381E08F9381E4CD
:1012F0008F930E9449078FEF809304018DB79EB7AB
:101300000B960FB6F8949EBF0FBE8DBF80916207FB
:101310008823F1F0809103018823D1F081E090E0EF
:101320009F938F9382E697E09F938F9381E08F93B3
:101330008F9382E48F930E944907109262072DB722
:101340003EB7295F3F4F0FB6F8943EBF0FBE2DBF8B
:101350008091BD038823E9F0809103018823C9F0BF
:1013600086E190E09F938F938EE797E09F938F9312
:1013700081E08F938F9380E58F930E9449071092AD
:10138000BD038DB79EB707960FB6F8949EBF0FBEEC
:101390008DBF08950F931F93DF93CF9300D0CDB7E8
:1013A000DEB78091C003882309F4E5C10E94A4063A
:1013B00080918B06823609F00DC180918C068137B1
:1013C00009F448C0823730F48B3459F0803709F083
:1013D00001C13CC0833709F493C0843709F0FAC0D7
:1013E00021C0E091C403F091C50380819181909365
:1013F000670480936604809166049091670420914D
:10140000680430916904845E9D4F821B930B68E6EB
:1014100071E00E948F57845B904090936B0480939F
:101420006A04D8C0E091C403F091C5038081918122
:10143000A281B3818093C8039093C903A093CA0388
:10144000B093CB038FEF80930501C4C081E08093FC
:10145000BD03C0C00091C4031091C503F801808191
:101460008F3F21F40E942303F8018083E091C4039D
:10147000F091C5038081882311F481E003C0863098
:1014800010F085E08083E091C403F091C50346E548
:1014900060EB77E080810E94B7038091030188238D
:1014A000E1F3E091C403F091C5038081898389E46D
:1014B0008A8386E590E09F938F9380EB97E09F93DC
:1014C0008F9321E030E03F932F93CE0102969F93BC
:1014D0008F933F932F93CE0101969F938F9383E039
:1014E0008F9381E08F9381E58F930E9449078DB799
:1014F0009EB70F960FB6F8949EBF0FBE8DBF6AC001
:10150000E091C403F091C50380818150853008F0DB
:1015100045C08181893409F041C0A0EBB7E0329623
:1015200086E501900D928150E1F7E091C403F091BE
:10153000C50346E560EB77E080810E948A036091F5
:10154000DB0770E080E090E024EC39E040E050E020
:101550000E9450576093950370939603809397036E
:10156000909398036091DC0770E080E090E00E9427
:1015700050576093990370939A0380939B039093C1
:101580009C03E091C403F091C50380810E943E0357
:101590000E94230389830E94D52801C0198280916B
:1015A00003018823E1F381E090E09F938F93CE01C4
:1015B00001969F938F9381E08F938F9383E58F9311
:1015C0000E944907EDB7FEB737960FB6F894FEBFF5
:1015D0000FBEEDBF80918C06873609F4C1C08836F6
:1015E00080F4813609F460C0823620F48B3409F02F
:1015F000BAC039C0823609F464C0843609F0B3C079
:1016000075C08C3609F49AC08D3620F4883609F0FE
:10161000AAC07FC0843721F0863709F0A4C09CC0DF
:10162000E091C403F091C50380819181A281B381CF
:101630008093C8039093C903A093CA03B093CB03CC
:10164000809103018823E1F31F92809106018F931B
:1016500084E58F930E9449078FEF809305010F90D7
:101660000F900F9080C0E091C403F091C50380817A
:1016700091819093670480936604809166049091B1
:1016800067042091680430916904845E9D4F821B39
:10169000930B68E671E00E948F57845B90409093B3
:1016A0006B0480936A045FC0E091C403F091C503AA
:1016B0008081809304018032A8F08FE1809304013F
:1016C00011C0ADE7B6E08091C4039091C5039C01C1
:1016D000F9018BE001900D928150E1F7809186062F
:1016E000809362078FEF809305013DC0E091C403B2
:1016F000F091C50380812AE0829FC001112490935C
:10170000080180930701892B71F181E08093BB036D
:101710002AC08FEF80930501E091C403F091C503C7
:10172000808190910C04892B80930C04882311F004
:101730001092BE0381E08093BA0315C08FEF8093AF
:101740000501E091C403F091C503808180930B04EF
:1017500081E08093B90307C081E08093BC0303C09C
:1017600081E08093B8031092C0031092C5031092D9
:10177000C4031092C6030F900F90CF91DF911F9179
:101780000F9108951F920F920FB60F9211242F936D
:101790003F934F935F936F937F938F939F93AF93F9
:1017A000BF93CF93DF93EF93FF938091C600809315
:1017B000BF038091BF030E94E5484091CD034639A5
:1017C00010F01092CC038091BF038D3009F05DC002
:1017D0008091CC03823009F058C01092CC03A42F22
:1017E000B0E0FD01E857F94F3081ED01C757D94FFF
:1017F00028818091D0039091D103831B9109821B92
:1018000091099F709093D1038093D0039C0196E03F
:10181000369527959A95E1F7235C2093CF03982F6F
:101820009F73935C9093CE038081281729F488815D
:10183000981711F491E006C08091C2038F5F8093E6
:10184000C20390E08091C003882309F06AC0992305
:1018500009F467C081E08093C0034F5F4093C303E6
:10186000A657B94F8DE08C9380918C06823509F094
:1018700058C02CE088E190E00FB6F894A8958093CA
:1018800060000FBE209360004CC08091CC0381307B
:10189000F9F0813020F0823009F041C024C08091FD
:1018A000BF03833239F48091C003882319F481E0A7
:1018B0008093CC038091BF0380938A0681E080935C
:1018C000CD038091BF038093D0031092D10329C030
:1018D00082E08093CC03E42FF0E08091BF03E657D1
:1018E000F94F808309C0E42FF0E08091BF03E657F1
:1018F000F94F8083463920F44F5F4093CD0302C0F7
:101900001092CC032091BF038091D0039091D1031A
:10191000820F911D9093D1038093D00302C0109247
:10192000CC03FF91EF91DF91CF91BF91AF919F9148
:101930008F917F916F915F914F913F912F910F9078
:101940000FBE0F901F901895982F809163078130DC
:1019500061F480910A04E82FF0E0EA5DFC4F908387
:101960008F5F80930A0481E00895892F0E94FF060B
:1019700008951F93182F04C080E30E94A40C1150F7
:101980001116D4F31F9108951F93182F04C080E2FD
:101990000E94A40C11501116D4F31F9108950F93B7
:1019A0001F93CF93DF938C01EB0108C0F8010F5F09
:1019B0001F4FE4918E2F0E94A40C21972097B1F71E
:1019C000DF91CF911F910F9108950F931F93CF93A4
:1019D000DF938C01EB0106C0F80181918F010E9419
:1019E000A40C21972097C1F7DF91CF911F910F9100
:1019F00008952F923F924F925F926F927F928F92B3
:101A00009F92AF92BF92CF92DF92EF92FF920F938D
:101A10001F93DF93CF93CDB7DEB7E5970FB6F8945A
:101A2000DEBF0FBECDBF2C969FAD2C972D964FAD30
:101A30002D972B968FAD2B9780936307EDE4AE2EF9
:101A4000B12CAC0EBD1E292F342FC9019DA78CA728
:101A50001EA61FA618AA19AA9E01245D3F4F3DABE2
:101A60002CAB0CA51DA502C00F5F1F4FF801F49011
:101A7000FF2019F0F5E2FF16B9F7B8012CA53DA536
:101A8000621B730B19F0C9010E94CF0CFF2009F4EF
:101A900052C2A8014F5F5F4F5DA74CA71982442433
:101AA0001BAA5FEF5AAB02C0C5015C01ECA5FDA506
:101AB000CF0101969DA78CA76491A42DB0E0A170E1
:101AC000B070653721F0862F80628837F1F4109767
:101AD00071F0F50120813181428153812EA73FA70A
:101AE00048AB59AB24E030E0A20EB31E0EC0F501A6
:101AF000808191819C0140E050E02EA73FA748AB38
:101B000059AB42E050E0A40EB51E603221F4898149
:101B1000882351F61AC0633211F458E05AC06A3271
:101B200021F06D3281F4C50109C0C5010296D501CD
:101B3000BC91BBABB7FFB9CFB195BBABE0E14E2ACF
:101B4000FFED4F22B2CF6B3211F46983ADCF6E320D
:101B500009F03AC0ECA5FDA59F012F5F3F4F3DA7BF
:101B60002CA784918A3221F0682F20E030E021C038
:101B7000C5010296D5014D915C9157FF02C04FEF10
:101B80005FEF4AAB92CFC90173E0880F991F7A9536
:101B9000E1F7220F331F280F391F260F311D205365
:101BA0003040ECA5FDA5AF014F5F5F4F5DA74CA78F
:101BB0006491862F80538A3030F3A90137FF02C029
:101BC0004FEF5FEF4AAB7DCF603329F444FC6CCF1D
:101BD00050E2452A69CF862F81538930E8F420E00E
:101BE00030E0C90143E0880F991F4A95E1F7220FC1
:101BF000331F280F391F260F311D20533040ECA50D
:101C0000FDA5CF0101969DA78CA76491862F8053D7
:101C10008A3038F32BAB55CF683619F494E0492A53
:101C200043CF6C3619F4A1E04A2A3ECF562EF50177
:101C3000B3E66B1741F422E030E0A20EB31E8081C0
:101C40008C83198225C134E4631739F044E66417A4
:101C500031F059E66517C1F502C081E0482A40FE1F
:101C600009C0A4E0B0E0AA0EBB1E208131814281F0
:101C700053810BC042E050E0A40EB51E80819181DB
:101C80009C01442737FD4095542F2EA73FA748AB12
:101C900059AB8EA59FA5A8A9B9A9B7FF11C02EA5BC
:101CA0003FA548A959A950954095309521953F4F9A
:101CB0004F4F5F4F2EA73FA748AB59AB3DE239834B
:101CC000562E1AE0312E80C04FE4641721F05FE6F3
:101CD000651731F402C081E0482AB8E03B2E73C09A
:101CE00090E7691791F4A2E0B0E0AA0EBB1E8081D4
:101CF00091819C0140E050E02EA73FA748AB59AB33
:101D000030E4432AA8E75A2E5CC06337E1F5D501D9
:101D1000CD90DC90C114D10489F4B8E2BC83EEE626
:101D2000ED83F5E7FE832CE62F83288739E2398798
:101D30001A86F4E0CF2ED12CCC0EDD1E4AA947FD29
:101D400010C0552747FD509560E070E0C6010E9425
:101D5000F054009771F0182F1C195AA951174CF024
:101D600009C0F60101900020E9F731971E2F1C19D8
:101D700001C01AA982E090E0A80EB91E1982E3E71B
:101D80005E2E40E08CC0653521F0653739F4562E63
:101D900002C091E0492A7AE0372E15C0683519F063
:101DA000683709F06FC043FE0BC02EA53FA548A9B8
:101DB00059A9211531054105510511F030E4432A97
:101DC000562E60E1362E19824AA947FD02C05FED0A
:101DD00045228EA59FA5A8A9B9A90097A105B1057F
:101DE00049F49AA9992331F45CE2C52ED12CCC0E8A
:101DF000DD1E44C04CE2C42ED12CCC0EDD1EEEA460
:101E0000FFA408A919A9632C772488249924C80160
:101E1000B701A40193010E94A2576A3020F430E375
:101E2000232E260E08C027E5222E260EA8E55A16D8
:101E300011F4BFED2B22F60122926F01C801B70108
:101E4000A40193010E94A257C901DA018EA79FA79E
:101E5000A8ABB9ABE614F7040805190518F07C0126
:101E60008D01D5CFF8E03F1649F443FE07C020E3CB
:101E7000221621F0D601E0E3EE936D011CA91C1996
:101E80004AA90DC0662309F456C06C831982562EE8
:101E900094E0C92ED12CCC0EDD1E40E011E0042FC1
:101EA000011B07FD00E08981882319F0812F8F5FD6
:101EB00006C046FC02C0812F02C0812F8E5F782EA3
:101EC000700EE42CFF2480E3882E912C8E209F201E
:101ED0008114910421F48BA987190E94C40C898173
:101EE000882329F061E070E0CE01019609C0E6FE8A
:101EF00009C0F0E3FA835B8262E070E0CE010296F3
:101F00000E94E50C20E28216910421F48BA9871926
:101F10000E94B90C802F0E94B90C612F772767FDB2
:101F20007095C6010E94E50CE4FE9BCD8BA9871934
:101F30000E94C40C96CDE5960FB6F894DEBF0FBE96
:101F4000CDBFCF91DF911F910F91FF90EF90DF9068
:101F5000CF90BF90AF909F908F907F906F905F9049
:101F60004F903F902F9008951F920F920FB60F92AF
:101F700011242F933F935F936F937F938F939F933E
:101F8000AF93BF938091DB03882329F08091DB031B
:101F900081508093DB038091E30381508093E303BE
:101FA0008F5F11F58091E1039091E203009729F092
:101FB00001979093E2038093E10389E08093E30328
:101FC000809110038F5F817080931003882319F430
:101FD00081E08093D6038091D4039091D50301963C
:101FE0009093D5038093D4038091D9039091DA0321
:101FF0000297B8F08091D9039091DA0301979093FA
:10200000DA038093D9038091D9039091DA03209168
:102010000B0330910C0382239323892B09F0A3C077
:1020200006C08FEF9FEF90930C0380930B0380917A
:1020300000018A3039F404C05A9A05C0479A03C097
:102040005A9801C04798349B0AC08091D703909159
:10205000D80301969093D8038093D7038AC08091C8
:10206000D7039091D803892B09F45FC08091D703DF
:102070009091D8038A56914008F057C02091D70319
:102080003091D8038091D7039091D80369E270E032
:102090000E947B57260F371F3093D8032093D70316
:1020A0008091D7039091D8030B9750F08091D7037C
:1020B0009091D8030A97909367048093660404C0B4
:1020C00010926704109266048FEF90E09093E20301
:1020D0008093E1038091D7039091D8038758904073
:1020E00090936704809366048091660490916704DE
:1020F00097FF0AC0809166049091670488599E4FAB
:1021000090936704809366048091660490916704BD
:102110008856914054F080916604909167048856E7
:102120009140909367048093660480916604909137
:1021300067042091680430916904845E9D4F821B7E
:10214000930B68E671E00E948F57845B90409093F8
:102150006B0480936A0481E08093DE031092D803BD
:102160001092D70306C0809100018A3009F066CF33
:1021700063CFBF91AF919F918F917F916F915F914D
:102180003F912F910F900FBE0F901F901895809147
:10219000D4039091D5030B969093E5038093E403C9
:1021A00082E085BD83EA84BD17BC88E788BD86E0F0
:1021B00086BD83EC8093B00084E08093B100E0E7BB
:1021C000F0E0808182608083EEE6F0E080818160D3
:1021D00080838AE08093B3001092B200089520912A
:1021E000D4033091D5032F5F3F4F280F391FC9010A
:1021F00008952091D4033091D503821B930B8070F6
:102200009078892F869508952091D4033091D50335
:102210002F5F3F4F280F391F8091D4039091D50332
:10222000A901481B590BCA0180709078892F8695A7
:1022300099F308952091D4033091D5032F5F3F4F38
:10224000280F391F4FEE02C040937A008091D403CB
:102250009091D503B901681B790BCB018070907800
:10226000892F869589F308951F920F920FB60F92CA
:1022700011248F939F938091090390910A03892BD6
:1022800011F05F9A01C05F9883E08093B000809165
:1022900070008E7F809370009F918F910F900FBE82
:1022A0000F901F9018951F920F920FB60F92112446
:1022B0002F933F934F935F936F937F938F939F934E
:1022C000AF93BF93CF93DF93EF93FF938091090375
:1022D00090910A03049709F088C08091AA0390E0C6
:1022E000880F991F40910D0350910E039A01220F00
:1022F000331F240F351F820F931F64E070E00E948C
:102300008F5770930E0360930D03EB01E09680915D
:10231000F60720912A0430912B0440912C0450910F
:102320002D0480FF0EC06091D20770E080E090E045
:102330000E94505720E030E440E050E00E94C45733
:1023400014C06091D20770E080E090E00E94505786
:1023500020E030E440E050E00E94C45750954095A2
:10236000309521953F4F4F4F5F4FC20FD31FD093F2
:10237000DD03C093DC032091DC033091DD03809109
:10238000D30743E0849FC00111242817390740F088
:102390008091D407849FC00111248217930720F4F1
:1023A0009093DD038093DC032091DC033091DD0307
:1023B00030934B0720934A07C9016FEF70E00E94EA
:1023C0007B578D9740F4235B3F4F3093DD03209381
:1023D000DC0383E101C080E680930F038091DC037E
:1023E00080958093B30083EC40C080910903909165
:1023F0000A03892B39F18091090390910A0304970C
:1024000008F52091DC033091DD032F3F310561F0A9
:1024100058F05F9A83E08093B0002F5F3040309394
:10242000DD032093DC0323C083E88093B000809118
:102430000F038093B30081E090E090930A038093B0
:10244000090315C08091090390910A03892B79F43F
:102450008091D50790E0880F991F880F991F90935E
:102460000A03809309035F9883E08093B000809112
:10247000090390910A03019790930A03809309033B
:10248000FF91EF91DF91CF91BF91AF919F918F918C
:102490007F916F915F914F913F912F910F900FBE60
:1024A0000F901F90189510927C008FEE80937A0009
:1024B00008951F920F920FB60F921124CF92DF92C0
:1024C000EF92FF920F931F932F933F934F935F933E
:1024D0006F937F938F939F93AF93BF93EF93FF93EC
:1024E00010927A00809106048F5F809306048150D9
:1024F000853009F486C0863090F4823009F440C0FB
:10250000833030F48823F1F0813009F09DC22FC070
:10251000833009F441C0843009F096C25AC0883033
:1025200009F4D5C0893038F4863009F483C0873087
:1025300009F08AC2AFC0893009F4E6C08A3009F0D8
:1025400083C2D9C18091780090917900909305045D
:102550008093040481E0809307048091FB039091B1
:10256000FC0301969093FC038093FB0371C280915E
:102570007800909179009093030480930204A5C0A1
:1025800080917800909179009093010480930004E9
:1025900084E0809307045CC24091110350911203C0
:1025A00080917800909179009A01220F331F240FB7
:1025B000351F63E070E00E947B57260F371F36956A
:1025C000279536952795309312032093110386E0C3
:1025D000E0CF209178003091790080912004909193
:1025E0002104821B930B909365078093640780916D
:1025F0006407909165079093ED038093EC0387E067
:10260000C8CF809178009091790020911E0430917C
:102610001F04821B930B9093700780936F07809128
:102620006F07909170079093EF038093EE031092E1
:1026300007040EC2809100018A3069F4809178000D
:10264000909179002091040430910504820F931F2A
:102650009695879519C040910404509105048431E2
:1026600069F4209178003091790088279927841B9C
:10267000950B821B930B81509C4F06C08091780074
:1026800090917900840F951F9093EB038093EA0358
:1026900081E07FCF809100012091020430910304FA
:1026A0008A3049F48091780090917900820F931FCD
:1026B0009695879506C08091780090917900820F59
:1026C000931F9093E9038093E80382E062CF8091A7
:1026D000000120910004309101048A3049F4809176
:1026E000780090917900820F931F9695879506C088
:1026F0008091780090917900820F931F9093E70367
:102700008093E60385E045CF609178007091790071
:10271000E0902404F09025040091260410912704F1
:10272000882777FD8095982F0E943956A801970138
:102730000E9435550E9406567093F1036093F00392
:102740008091F0039091F10302970CF43EC06091E8
:10275000240470912504809126049091270420E0A0
:1027600030E84BE354E40E949A5588230CF078C07B
:10277000609124047091250480912604909127048F
:102780002AE037ED43EA5CE30E9436556093240467
:102790007093250480932604909327048091A904C4
:1027A0009091AA04845F914008F05AC0609124047B
:1027B0007091250480912604909127042DEC3CEC27
:1027C0004CEC5DE30E94365543C08091F00390913C
:1027D000F1038F5F9F4F0CF043C060912404709110
:1027E0002504809126049091270420E030E849E0F8
:1027F00054E40E94E95618169CF5609124047091E7
:10280000250480912604909127042AE037ED43EABD
:102810005CE30E94355560932404709325048093F3
:102820002604909327048091A9049091AA04845FC0
:102830009140B0F4609124047091250480912604A5
:10284000909127042DEC3CEC4CEC5DE30E94355557
:1028500060932404709325048093260490932704A6
:1028600081E08093F70380917800909179009093B4
:10287000670780936607209162043091630440915A
:102880006404509165048091F0039091F103AA27AC
:1028900097FDA095BA2F820F931FA41FB51F809399
:1028A000620490936304A0936404B0936504E09081
:1028B0006204F090630400916404109165046091D7
:1028C000620470916304809164049091650420E037
:1028D00034E040E050E00E94C457E21AF30A040BCF
:1028E000150BE0926204F092630400936404109369
:1028F000650483E04ECE8091740790917507209116
:10290000780030917900820F931F90937507809320
:10291000740780916C078F5F80936C0780916C07C0
:10292000853008F491C0809178009091790090935F
:1029300018038093170310926C076091F90370914C
:10294000FA038091F803992787FD90952FEF30E0E7
:10295000829F6001839FD00C929FD00C1124209104
:1029600068073091690780917407909175074091CD
:10297000870450918804281B390B241B350B2C0D20
:102980003D1D8091A10390E0AC01249FC001259FD3
:10299000900D349F900D11249B0153E0220F331FA3
:1029A0005A95E1F7261B370B820F931F68E070E002
:1029B0000E948F577093FA036093F9032091740774
:1029C00030917507E0901303F09014030091150304
:1029D00010911603C801B701660F771F881F991F52
:1029E0006E0D7F1D801F911F442737FD4095542F8A
:1029F000620F731F841F951F24E030E040E050E019
:102A00000E94C457C901DA01809313039093140301
:102A1000A0931503B09316032091680730916907BE
:102A20008091130390911403A0911503B0911603A4
:102A3000C20ED31EC81AD90AD0928804C092870445
:102A400010927507109274071092070410920604F2
:102A50008091070480937C0080910604882319F0FC
:102A60008FEE80937A00FF91EF91BF91AF919F918C
:102A70008F917F916F915F914F913F912F911F9116
:102A80000F91FF90EF90DF90CF900F900FBE0F90BF
:102A90001F901895BF92CF92DF92EF92FF920F9303
:102AA0001F931092FD031092FE031092FF030CE897
:102AB000FF24F39498E0B92E8AE0D82E15EFE12E8A
:102AC000BFEECB2E05C0133019F40B3008F009E02F
:102AD0008091E6039091E7038C5F934024F480910A
:102AE000190381500CC08091E6039091E703875051
:102AF000944014F411E006C0809119038F5F809315
:102B0000190310E08091E8039091E9038C5F9340F2
:102B100024F480911A0381500AC08091E8039091B7
:102B2000E9038750944034F080911A038F5F8093BB
:102B30001A0301C01F5F8091EA039091EB038C5F41
:102B4000934024F480911B0381500AC08091EA03D2
:102B50009091EB038750944034F080911B038F5F7A
:102B600080931B0301C01F5FB0920D040E94061DDD
:102B7000809119038A3020F4F092FD03D09219035A
:102B800080911903863F20F0F092FD03E092190333
:102B900080911A038A3020F4F092FE03D0921A0337
:102BA00080911A03863F20F0F092FE03E0921A0310
:102BB00080911B038A3020F4F092FF03D0921B0314
:102BC00080911B03863F20F0F092FF03E0921B03ED
:102BD00080910D048823E1F710926C07C0927A006F
:102BE00080916C078823E1F30A3020F48AE090E0BA
:102BF0000E941A11015009F066CF86E490E00E940D
:102C00001A111F910F91FF90EF90DF90CF90BF901E
:102C10000895EF92FF920F931F93CF93DF93F9994B
:102C2000FECF23E0E22E20E0F22EF2BCE1BCF89AC7
:102C300080B5C82FD0E0C531D10508F02A97C7BDAF
:102C40001092F80384E690E00E941A118091170315
:102C50009091180382559340C8F4C0E0D0E016C0AC
:102C6000C7BD82E390E00E941A111F930F931F9239
:102C70000E94F90C80911703909118030F900F9008
:102C80000F908255934038F0219602C008EF11E072
:102C9000CA3FD10528F38C2FF999FECF1FBAF2BC99
:102CA000E1BC80BD0FB6F894FA9AF99A0FBE8093F2
:102CB00071078CE291E00E941A11DF91CF911F9170
:102CC0000F91FF90EF900895E6E2F3E080E28193A8
:102CD00093E0E637F907D9F708951F9340917603FB
:102CE00080910B04481710F440930B0480910C045E
:102CF000282F30E080FF0AC090910B04992321F027
:102D0000915090930B0402C040930B0421FF0AC022
:102D100090910B04941719F410920B0403C09F5F59
:102D200090930B04237030702330310511F410920E
:102D30000B04E6E2F3E080E2819393E0E637F907E3
:102D4000D9F780910B04282F30E08A3040F481E1DC
:102D500080930A043F932F9383E295E007C080E1BC
:102D600080930A043F932F938EE195E09F938F9376
:102D700081E08F930E94F90C0F900F900F900F90AD
:102D80000F9010910B04153009F4FBC1163090F42C
:102D9000123009F4C8C0133030F4112309F1113096
:102DA00009F097C465C0133009F413C1143009F059
:102DB00090C463C1183009F47AC3193038F416305E
:102DC00009F403C3173009F084C44DC31A3009F461
:102DD000EDC31A3008F4A9C31B3009F07AC427C424
:102DE00010920A048EE095E09F938F9311E01F9359
:102DF0000E94F90C84E180930A042091000188E686
:102E000090E09F938F9387E490E09F938F931F921E
:102E10001F92822F6AE00E946F57892F90E09F9344
:102E20008F93822F0E946F5790E09F938F9389EF2B
:102E300094E09F938F931F930E94F90C88E28093F4
:102E40000A040E94230390E09F938F938CEE94E0FA
:102E50009F938F931F930E94F90C8CE380930A0435
:102E60008CED94E09F938F931F930E94F90C2DC4D7
:102E70008091B80780FF3AC010920A0480918704BD
:102E8000909188049F938F938DEC94E09F938F9300
:102E90001F930E94F90C84E180930A0480918904B5
:102EA00090918A049F938F938EEB94E09F938F93DE
:102EB0001F930E94F90C88E280930A048091170303
:102EC000909118039F938F938FEA94E09F938F9331
:102ED0001F930E94F90C8CE380930A048091710780
:102EE00090E09F938F9380EA94E05AC384E18093AB
:102EF0000A0489E994E09F938F931F930E94F90C31
:102F000088E280930A048BE894E09F938F931F9349
:102F10000E94F90C8DB79EB706960FB6F8949EBF27
:102F20000FBE8DBFDBC310920A0481E894E09F932B
:102F30008F9311E01F930E94F90C84E180930A049F
:102F400060912A0470912B0480912C0490912D049F
:102F500020E034E040E050E00E94C4575F934F937C
:102F60003F932F9382E794E09F938F931F930E9448
:102F7000F90C88E280930A04609132047091330462
:102F8000809134049091350420E034E040E050E03A
:102F90000E94C4575F934F933F932F9383E694E02F
:102FA0009F938F931F930E94F90C8CE380930A04E4
:102FB00080916604909167049F938F9384E594E0D9
:102FC0009F938F931F930E94F90C8DB79EB74696DF
:102FD000A4CF10920A0480918207909183072091D8
:102FE0008007309181079F938F933F932F9384E4C1
:102FF00094E09F938F9311E01F930E94F90C84E15A
:1030000080930A0480918607909187072091840716
:10301000309185079F938F933F932F9384E394E0A0
:103020009F938F931F930E94F90C88E280930A0468
:1030300080918A0790918B072091880730918907AA
:103040009F938F933F932F9384E294E09F938F936A
:103050001F930E94F90C8CE380930A0480918E07E1
:1030600090918F0720918C0730918D079F938F93BC
:103070003F932F9384E194E07BC010920A04E09187
:10308000B107F0E0EE0FFF1FE258F84F20813181C9
:10309000E091B007F0E0EE0FFF1FE258F84F80819B
:1030A00091813F932F939F938F9384E094E09F931C
:1030B0008F9311E01F930E94F90C84E180930A041E
:1030C000E091B307F0E0EE0FFF1FE258F84F2081C8
:1030D0003181E091B207F0E0EE0FFF1FE258F84FA8
:1030E000808191813F932F939F938F9384EF93E0FF
:1030F0009F938F931F930E94F90C88E280930A0498
:10310000E091B507F0E0EE0FFF1FE258F84F208185
:103110003181E091B407F0E0EE0FFF1FE258F84F65
:10312000808191813F932F939F938F9384EE93E0BF
:103130009F938F931F930E94F90C8CE380930A0452
:10314000E091B707F0E0EE0FFF1FE258F84F208143
:103150003181E091B607F0E0EE0FFF1FE258F84F23
:10316000808191813F932F939F938F9384ED93E080
:103170009F938F931F930E94F90C8DB79EB74C9627
:10318000CCCE10920A0486EC93E09F938F9311E0CB
:103190001F930E94F90C809100010F900F900F90E7
:1031A0008A3009F044C084E180930A048091E603E8
:1031B0009091E70320911404309115043F932F93CD
:1031C000821B930B9F938F9387EB93E09F938F9337
:1031D0001F930E94F90C88E280930A048091E8030F
:1031E0009091E90320911604309117043F932F9397
:1031F000821B930B9F938F9388EA93E09F938F9307
:103200001F930E94F90C8CE380930A0480911804A8
:10321000909119042091EA033091EB039F938F93CF
:10322000821B930B9F938F9389E993E058C08B3057
:1032300019F0843109F05CC084E180930A04E091C4
:103240001404F09115042091E6033091E703CF01B7
:1032500062E070E00E948F577F936F932E1B3F0BAD
:103260003F932F938AE893E09F938F9311E01F93EE
:103270000E94F90C88E280930A04E0911604F09110
:1032800017042091E8033091E903CF0162E070E078
:103290000E948F577F936F932E1B3F0B3F932F936B
:1032A0008BE793E09F938F931F930E94F90C8CE31D
:1032B00080930A042091180430911904E091EA03E4
:1032C000F091EB03C90162E070E00E948F577F9399
:1032D0006F932E1B3F0B3F932F938CE693E09F93AE
:1032E0008F931F930E94F90C8DB79EB7459615CE0C
:1032F0008D3009F0F3C184E180930A04E091140455
:10330000F09115042091E6033091E70380911903B1
:1033100090E09F938F93CF0162E070E00E948F57FF
:103320007F936F932E1B3F0B3F932F9388E593E082
:103330009F938F931F930E94F90C88E280930A0455
:10334000E0911604F09117042091E8033091E9030D
:1033500080911A0390E09F938F93CF0162E070E019
:103360000E948F577F936F932E1B3F0B3F932F939A
:1033700084E493E09F938F931F930E94F90C8CE356
:1033800080930A042091180430911904E091EA0313
:10339000F091EB0380911B0390E09F938F93C90101
:1033A00062E070E00E948F577F936F932E1B3F0B5C
:1033B0003F932F9380E393E09F938F931F930E94FB
:1033C000F90C8DB79EB74B96A8CD10920A0483E2F4
:1033D00093E09F938F9311E01F930E94F90C84E177
:1033E00080930A042091EE033091EF0380911E0434
:1033F00090911F049F938F933F932F9384E193E0C9
:103400009F938F931F930E94F90C88E280930A0484
:103410002091EC033091ED038091200490912104E0
:103420009F938F933F932F9385E093E09F938F9388
:103430001F930E94F90C8CE380930A04609124048A
:103440007091250480912604909127040E940656CD
:103450007F936F9380912408909125089F938F9379
:1034600086EF92E02DC184E180930A0480911103DC
:10347000909112039F938F9387EE92E09F938F9387
:1034800011E01F930E94F90C88E280930A04809156
:103490007D0490E09F938F9388ED92E09F938F93AC
:1034A0001F930E94F90C8DB79EB70A9636CD1092E5
:1034B0000A0489EC92E09F938F9311E01F930E947E
:1034C000F90C84E180930A0480916A0490916B0462
:1034D0009F938F938AEB92E09F938F931F930E9409
:1034E000F90C88E280930A04809166049091670445
:1034F0009F938F938BEA92E09F938F931F930E94E9
:10350000F90C8CE380930A0480916804909169041B
:103510009F938F938CE992E09F938F931F930E94C8
:10352000F90C8DB79EB74296F8CC10920A048091A0
:103530007504909176049F938F9380E992E09F9316
:103540008F9311E01F930E94F90C84E180930A0489
:1035500080917704909178049F938F9384E892E010
:103560009F938F931F930E94F90C88E280930A0423
:103570008091790490917A049F938F9388E792E0E9
:103580009F938F931F930E94F90C8CE380930A04FE
:1035900080917B0490917C049F938F938CE692E0C2
:1035A0009F938F931F930E94F90C3DC010920A04C1
:1035B00084E692E09F938F9311E01F930E94F90C91
:1035C00084E180930A048091AA0390E09F938F93F3
:1035D00086E592E09F938F931F930E94F90C88E2F7
:1035E00080930A048091DC039091DD039F938F9375
:1035F00088E492E09F938F931F930E94F90C8CE3D1
:1036000080930A048091D40790E09F938F938091D8
:10361000D30790E09F938F938AE392E09F938F93D9
:103620001F930E94F90C8DB79EB7449676CC1092EA
:103630000A048AE292E09F938F9311E01F930E9405
:10364000F90C84E180930A0480918106992787FD13
:1036500090959F938F9380918006992787FD9095F1
:103660009F938F938AE192E09F938F931F930E9481
:10367000F90C88E280930A0480918206992787FDDD
:1036800090959F938F938091830690E09F938F9363
:103690008AE092E09F938F931F930E94F90C8CE332
:1036A00080930A048091870690E09F938F93809186
:1036B0008406992787FD90959F938F938AEF91E0D9
:1036C0009F938F931F930E94F90C8DB79EB74896D6
:1036D00024CC11501093760310920B0410920C041A
:1036E0001F910895EF92FF920F931F93CF93DF9353
:1036F0008C01EB019C0197FF04C022273327281B74
:10370000390BCE01D7FF04C0882799278C1B9D0B4E
:10371000821793073CF4CE01E8018C01B1E0EB2E57
:10372000F12C02C0EE24FF24209741F4011511056D
:1037300029F461E070E080E090E025C0B8018827BE
:1037400077FD8095982F28EE33E040E050E00E940E
:1037500050579E01442737FD4095542F0E94C4576F
:10376000A90137FF03C0509541955F4FBA018827E3
:1037700077FD8095982F6D3021E0720720E0820759
:1037800020E0920704F524E630E040E050E00E949B
:1037900050572CE031E040E050E00E94C457CA018D
:1037A000B901A4E0660F771F881F991FAA95D1F76A
:1037B000621B730B840B950B24E630E040E050E075
:1037C0000E94C45753C0633442E0740740E084074A
:1037D00040E0940734F524E630E040E050E00E94F9
:1037E0005057605B78468040904026E331E040E0EF
:1037F00050E00E94C457CA01B901F4E0660F771F78
:10380000881F991FFA95D1F7621B730B840B950BD8
:1038100024E630E040E050E00E94C457215F3F4F73
:1038200025C022E330E040E050E00E945057645E43
:1038300070478040904026EA31E040E050E00E942E
:10384000C457CA01B901E4E0660F771F881F991FAA
:10385000EA95D1F7621B730B840B950B22E330E0E2
:1038600040E050E00E94C457225E3F4FEF2831F401
:103870008AE590E0AC01421B530B9A0117FD03C08F
:10388000D7FF06C002C0D7FD03C0309521953F4F3A
:10389000C901DF91CF911F910F91FF90EF90089593
:1038A0009C0137FF04C088279927821B930B8856F9
:1038B000914034F0C90168E671E00E948F579C0185
:1038C00037FD03C061E070E005C0309521953F4FA2
:1038D0006FEF7FEFC9018B5590408A35910538F421
:1038E00084EB90E0AC01421B530B9A010FC0C9015D
:1038F000855B90408A35910518F4245B30400FC0F9
:10390000C9018F5091408A35910518F041E050E08F
:1039100008C088E691E0AC01421B530B9A014FEFBF
:103920005FEFF901EE0FFF1FE85DFA4F859194916B
:10393000469F9001479F300D569F300D1124A901DD
:10394000489F9001499F300D589F300D1124C901A7
:1039500008952AE530E0A901481B590BCA010E94CD
:10396000501C0895EF92FF920F931F93CF93DF9314
:103970008C01EB01BC0197FF04C066277727681B09
:10398000790B9E01D7FF04C0222733272C1B3D0B48
:103990002617370754F4CA010E94501C7C01B80155
:1039A000882777FD8095982F09C0CA010E94A91C1D
:1039B0007C01BE01882777FD8095982F28EE33E0A3
:1039C00040E050E00E9450570027F7FC0095102F70
:1039D000A80197010E94C457C90137FF03C0909501
:1039E00081959F4F9C01442737FD4095542FB90185
:1039F000CA01DF91CF911F910F91FF90EF90089531
:103A00001092B9008AE28093B800089585EA809305
:103A1000BC0080E0089584E98093BC0008954CEBDD
:103A200050E084E9DA018C9310920D042BEB30E026
:103A3000F901808110920E0480E88C931092BD00F1
:103A40001092BA001082E9EBF0E01082A8EBB0E02F
:103A50001C9210828AE28C9385EADA018C931082A0
:103A6000F901108285E88C9308951092B900809333
:103A7000BB0085E88093BC0080E008951F920F9200
:103A80000FB60F9211248F939F93EF93FF93809122
:103A90000D048F5F80930D048150E82FF0E0E73133
:103AA000F10508F093C0E85CFF4FEE0FFF1F059093
:103AB000F491E02D099480910E0490E08996880F8E
:103AC000991F0CC080910E048F5F80930E0481506B
:103AD00029C0833009F07AC080914C081092B90057
:103AE0008093BB0085E88093BC0070C084E980931C
:103AF000BC0080910E04843018F410920D044AC06A
:103B000010920E0447C080910F04880F8D5AE6CFA3
:103B10008091BB00E0910F04F0E0EA58F84F8083F9
:103B200080910F04813041F0813018F0823089F6A5
:103B300006C080910B08D2CF80911408CFCF80911E
:103B40003F08CCCF80910F049091BB00E82FF0E0AC
:103B5000EA58F84F94838F5F80930F04843058F1B4
:103B600010920F0428C01092B90080E1B9CF809163
:103B70001903B4CF1092B90082E1B2CF80911A0339
:103B8000ADCF84E98093BC008AE090E090939203EB
:103B90008093910385EAA7CF1092B90088E9A0CF5E
:103BA0001092B90084E19CCF80911B0397CF1092B3
:103BB000B90080E895CF84E98093BC008AE090E06A
:103BC000909392038093910310920D048091BC0016
:103BD00080688093BC00FF91EF919F918F910F902F
:103BE0000FBE0F901F90189583EC80938100EFE635
:103BF000F0E0808180628083109219041092180492
:103C000010921704109216041092150410921404C6
:103C100008951F920F920FB60F9211240F931F93C6
:103C20002F933F934F935F936F937F938F939F93C4
:103C3000AF93BF93CF93DF93EF93FF9320918600D1
:103C4000309187008091120490911304281B390B46
:103C500080918600909187009093130480931204C2
:103C6000C9018D5494400091100410911104835F98
:103C70009A4160F40430110514F01092770381E04A
:103C800090E090931104809310048AC00A301105CB
:103C90000CF086C0C9018B5F9040845B914008F0B6
:103CA00068C0E901C25DD140F801EE0FFF1FE25884
:103CB000F84F808191819E01281B390BC90137FF84
:103CC00003C0909581959F4F06974CF480917D0499
:103CD000883C28F480917D04865F80937D04F80100
:103CE000EE0FFF1FE258F84F20813181C901880F84
:103CF000991F820F931F8C0F9D1F64E070E00E943C
:103D00008F579B01CE010196861797071CF421500F
:103D1000304006C021976C177D0714F42F5F3F4F8A
:103D200080917D04E801CC0FDD1F833CB8F0FE01DB
:103D3000E258F84F80819181A901481B590BCA01B3
:103D400063E070E00E948F57CB01880F991F860FA8
:103D5000971FCC56D84F9983888304C0CC56D84F30
:103D600019821882F801EE0FFF1FE258F84F3183D5
:103D70002083F8013196F0931104E0931004E530AC
:103D8000F10511F45D9A06C05D98E630F10511F475
:103D90005C9A05C05C98379711F45B9A01C05B98F8
:103DA000FF91EF91DF91CF91BF91AF919F918F9153
:103DB0007F916F915F914F913F912F911F910F9143
:103DC0000F900FBE0F901F90189581E08093B00761
:103DD00082E08093B10783E08093B20784E0809310
:103DE000B30785E08093B40786E08093B50787E04A
:103DF0008093B60788E08093B70708952F923F928B
:103E00004F925F926F927F928F929F92AF92BF92EA
:103E1000CF92DF92EF92FF920F931F93DF93CF9396
:103E2000CDB7DEB729970FB6F894DEBF0FBECDBF72
:103E30002091EA033091EB038091180490911904CA
:103E4000821B930B90935C0880935B082091EA039C
:103E50003091EB038091390890913A08821B930BC3
:103E60009093AD078093AC078091E8039091E903AC
:103E70002091160430911704821B930B90930A082B
:103E8000809309088091E6039091E7032091140440
:103E900030911504821B930B90931608809315089C
:103EA0006091EE037091EF03882777FD8095982F3E
:103EB0002CE030E040E050E00E9450579B01AC0104
:103EC0006091500870915108882777FD8095982F50
:103ED000620F731F841F951F22E030E040E050E026
:103EE0000E94C45730935108209350086091EC030E
:103EF0007091ED03882777FD8095982F2CE030E0B6
:103F000040E050E00E9450579B01AC01609169086D
:103F100070916A08882777FD8095982F620F731F2C
:103F2000841F951F22E030E040E050E00E94C4571B
:103F300030936A08209369086091F0037091F1034F
:103F4000882777FD8095982F2091240830912508A7
:103F5000442737FD4095542F620F731F841F951F10
:103F600022E030E040E050E00E94C4573093250842
:103F7000209324082091EE033091EF03C901880FAC
:103F8000991F820F931F880F991F880F991FAA27C7
:103F900097FDA095BA2F20913A0430913B044091AF
:103FA0003C0450913D04280F391F4A1F5B1F20938A
:103FB0003A0430933B0440933C0450933D042091D9
:103FC000EC033091ED03C901880F991F820F931FF5
:103FD000880F991F880F991FAA2797FDA095BA2FC0
:103FE00020913E0430913F0440914004509141049F
:103FF000280F391F4A1F5B1F20933E0430933F0454
:1040000040934004509341042091EE033091EF031C
:104010008091320890913308820F931F9093330858
:10402000809332082091EC033091ED0380915E087B
:1040300090915F08820F931F90935F0880935E08B2
:1040400080912204909123040196909323048093FD
:104050002204E0906607F0906707A0902404B090D7
:104060002504C0902604D0902704609142047091EA
:10407000430480914404909145040E9439563B01C9
:104080004C010027F7FC0095102FC801B7010E94D2
:104090003956A60195010E9435559B01AC01C4011A
:1040A000B3010E9436550E940656609342047093F5
:1040B0004304809344049093450480915B0890915D
:1040C0005C085C01CC24B7FCC094DC2C80916508B2
:1040D00090916608A0916708B0916808A80EB91E73
:1040E000CA1EDB1EA0926508B0926608C0926708DF
:1040F000D092680820915B0830915C08442737FD16
:104100004095542F80916F0890917008A09171088C
:10411000B0917208820F931FA41FB51F80936F0880
:1041200090937008A0937108B093720820915B0877
:1041300030915C08442737FD4095542F8091280822
:1041400090912908A0912A08B0912B08820F931F03
:10415000A41FB51F8093280890932908A0932A08CC
:10416000B0932B0880915B0890915C089C014427D8
:1041700037FD4095542F80915A0490915B04A09193
:104180005C04B0915D04280F391F4A1F5B1F2E830A
:104190003F834887598720935A0430935B044093A8
:1041A0005C0450935D0438E7A31637E1B30637E0AB
:1041B000C30630E0D30684F088E898EEA8EFBFEF9E
:1041C000A80EB91ECA1EDB1EA0926508B092660832
:1041D000C0926708D092680880916508909166083F
:1041E000A0916708B0916808B7FF0CC08858984E36
:1041F000A84FBF4F8093650890936608A093670807
:10420000B093680890918F049D83992309F094C01E
:1042100080919004882309F08FC08091B80786FFB1
:104220008BC06091AC077091AD07E0909D04FF24B6
:1042300000E010E0882777FD8095982F20914A04B0
:1042400030914B0440914C0450914D040E945057C2
:1042500020E038E040E050E00E94C457CA01B901B4
:10426000A80197010E94505720E030E140E050E063
:104270000E94C457D22EC32EB42EA52E2093EF0435
:104280003093F0044093F1045093F2046091AC0732
:104290007091AD07882777FD8095982F2091520463
:1042A0003091530440915404509155040E9450574A
:1042B00020E038E040E050E00E94C457CA01B90154
:1042C000A80197010E94505720E030E140E050E003
:1042D0000E94C457B901FA012093EB047093EC04D7
:1042E0004093ED04F093EE042D2D3C2D4B2D5A2DD3
:1042F000C901DA01B7FF07C0B095A09590958195E7
:104300009F4FAF4FBF4F81389105A105B10584F490
:10431000CB01DF01B7FF07C0B095A09590958195BF
:104320009F4FAF4FBF4F81389105A105B105A4F054
:1043300081E080936E0410C01092EB041092EC04A4
:104340001092ED041092EE041092EF041092F0041B
:104350001092F1041092F2048091090890910A08D9
:104360002091EF043091F0044091F1045091F20457
:1043700029833A834B835C83820F931F90930A08AF
:10438000809309080091090810910A086090EB04D5
:104390007090EC048090ED049090EE0480919E0467
:1043A000282E332444245524C201B101A4019301D1
:1043B0000E94505720E032E040E050E00E94C45795
:1043C000020F131F10930A0800930908209109088F
:1043D00030910A08442737FD4095542F80915604A8
:1043E00090915704A0915804B0915904820F931FE3
:1043F000A41FB51F8093560490935704A0935804AC
:10440000B09359048091090890910A0820918B0477
:1044100030918C04821B930BAA2797FDA095BA2F8D
:10442000209152043091530440915404509155040A
:10443000820F931FA41FB51F8093520490935304BF
:10444000A0935404B0935504A0909903B0909A039C
:10445000C0909B03D0909C03A816B906CA06DB0641
:10446000C4F488EA91E6A0E0B0E08A199B09AC099F
:10447000BD098093520490935304A0935404B093C5
:1044800055048093560490935704A0935804B09316
:10449000590422273327A9012A193B094C095D0930
:1044A0008091520490915304A0915404B09155040A
:1044B00082179307A407B507B4F4D601C501885A3B
:1044C0009146A040B0408093520490935304A0932F
:1044D0005404B09355048093560490935704A093CA
:1044E0005804B09359048091E8039091E9030F9721
:1044F00034F488E19CEF90930A0880930908809136
:10450000E8039091E903079734F480E398EF9093E0
:104510000A0880930908E09000013AE0E316A9F444
:104520008091E8039091E903835F934034F088EE33
:1045300093E090930A08809309088091E803909192
:10454000E9038A5F9340DCF014C08091E803909106
:10455000E903855E974034F088EE93E090930A0873
:10456000809309088091E8039091E903835F974065
:1045700034F080ED97E090930A08809309088091C9
:10458000150890911608861997099093160880933C
:1045900015080091150810911608C201B101298172
:1045A0003A814B815C810E94505720E032E040E02C
:1045B00050E00E94C45750954095309521953F4F4B
:1045C0004F4F5F4F020F131F1093160800931508EB
:1045D0002091150830911608442737FD4095542F37
:1045E00080914E0490914F04A0915004B0915104D9
:1045F000820F931FA41FB51F80934E0490934F0406
:10460000A0935004B093510480911508909116081E
:1046100020918D0430918E04821B930BAA2797FD65
:10462000A095BA2F20914A0430914B0440914C043C
:1046300050914D04820F931FA41FB51F80934A040D
:1046400090934B04A0934C04B0934D04A090950319
:10465000B0909603C0909703D0909803A816B9061F
:10466000CA06DB06C4F488EA91E6A0E0B0E08A1945
:104670009B09AC09BD0980934A0490934B04A09315
:104680004C04B0934D0480934E0490934F04A09338
:104690005004B093510422273327A9012A193B095A
:1046A0004C095D0980914A0490914B04A0914C04FF
:1046B000B0914D0482179307A407B507B4F4D6014F
:1046C000C501885A9146A040B04080934A04909317
:1046D0004B04A0934C04B0934D0480934E049093EC
:1046E0004F04A0935004B09351048091E60390913D
:1046F000E7030F9734F488E19CEF909316088093BA
:1047000015088091E6039091E703079734F480E35E
:1047100098EF9093160880931508EAE0EE16A9F436
:104720008091E6039091E703835F934034F088EE35
:1047300093E090931608809315088091E60390917A
:10474000E7038A5F9340DCF014C08091E603909108
:10475000E703855E974034F088EE93E09093160867
:10476000809315088091E6039091E703835F97405B
:1047700034F080ED97E090931608809315088FEE43
:1047800080937A008E819F81A885B98580934604A5
:1047900090934704A0934804B093490480914A043D
:1047A00090914B04A0914C04B0914D0480932A0445
:1047B00090932B04A0932C04B0932D048091520469
:1047C00090915304A0915404B09155048093320405
:1047D00090933304A0933404B093350480914E0435
:1047E00090914F04A0915004B091510480932E04F5
:1047F00090932F04A0933004B09331048091560419
:1048000090915704A0915804B091590480933604B4
:1048100090933704A0933804B09339048091B8077B
:1048200087FF63C09D81992309F05FC08091900448
:10483000882309F05AC08091150890911608893C88
:1048400091055CF0209115083091160880911508AB
:1048500090911608885C904011C080911508909145
:10486000160888539F4FA4F420911508309116081C
:10487000809115089091160888539F4F880F991FB3
:10488000880F991F820F931F909316088093150825
:104890008091090890910A08893C91055CF020916B
:1048A000090830910A088091090890910A08885CEB
:1048B000904011C08091090890910A0888539F4F39
:1048C000A4F42091090830910A0880910908909178
:1048D0000A0888539F4F880F991F880F991F820FCE
:1048E000931F90930A08809309088091B407E82FDA
:1048F000F0E0EE0FFF1FE258F84F80819181209188
:1049000075043091760483599F4F821793071CF0EA
:104910002F5F3F4F0CC08081918182599F4F82173A
:1049200093074CF42115310531F02150304030937C
:104930007604209375048091B507E82FF0E0EE0F20
:10494000FF1FE258F84F80819181209177043091C8
:10495000780483599F4F821793071CF02F5F3F4FB6
:104960000CC08081918182599F4F821793074CF42C
:104970002115310531F021503040309378042093D7
:1049800077048091B607E82FF0E0EE0FFF1FE258A2
:10499000F84F808191812091790430917A04835974
:1049A0009F4F821793071CF02F5F3F4F0CC08081F1
:1049B000918182599F4F821793074CF4211531053D
:1049C00031F02150304030937A0420937904809163
:1049D000B707E82FF0E0EE0FFF1FE258F84F808195
:1049E000918120917B0430917C0483599F4F8217E1
:1049F00093071CF02F5F3F4F0CC08081918182593B
:104A00009F4F821793074CF42115310531F0215047
:104A1000304030937C0420937B0480917504909106
:104A2000760497FF05C010927604109275040AC0B0
:104A30008F3F910539F034F08FEF90E0909376043A
:104A400080937504809177049091780497FF05C056
:104A500010927804109277040AC08F3F910539F0C4
:104A600034F08FEF90E090937804809377048091F6
:104A7000790490917A0497FF05C010927A041092FD
:104A800079040AC08F3F910539F034F08FEF90E040
:104A900090937A048093790480917B0490917C04B4
:104AA00097FF05C010927C0410927B040AC08F3FD0
:104AB000910539F034F08FEF90E090937C0480936F
:104AC0007B0429960FB6F894DEBF0FBECDBFCF9101
:104AD000DF911F910F91FF90EF90DF90CF90BF90EB
:104AE000AF909F908F907F906F905F904F903F908E
:104AF0002F9008958091BB078B3F98F08B3F19F45E
:104B0000809175040EC08C3F19F48091770409C020
:104B10008D3F19F48091790404C08E3F21F4809177
:104B20007B048093A2038091BA078B3F98F08B3F60
:104B300019F4809175040EC08C3F19F480917704AC
:104B400009C08D3F19F48091790404C08E3F21F48F
:104B500080917B048093A1038091A103882319F4A1
:104B60001092A10305C0843618F084E68093A10357
:104B70008091BC078B3F98F08B3F19F480917504AE
:104B80000EC08C3F19F48091770409C08D3F19F451
:104B90008091790404C08E3F21F480917B0480933E
:104BA000A3038091A303882319F41092A30305C0E3
:104BB000843618F084E68093A3038091BE078B3F70
:104BC00098F08B3F19F4809175040EC08C3F19F456
:104BD0008091770409C08D3F19F48091790404C055
:104BE0008E3F21F480917B048093A4038091C507BC
:104BF0008B3F98F08B3F19F4809175040EC08C3F69
:104C000019F48091770409C08D3F19F480917904DB
:104C100004C08E3F21F480917B048093A503809192
:104C2000C6078B3F98F08B3F19F4809175040EC036
:104C30008C3F19F48091770409C08D3F19F480915D
:104C4000790404C08E3F21F480917B048093A603F5
:104C50008091A6038B3010F48AE002C08F3F11F4DC
:104C60008093A6038091C7078B3F98F08B3F19F480
:104C7000809175040EC08C3F19F48091770409C0AF
:104C80008D3F19F48091790404C08E3F21F4809106
:104C90007B048093A7038091CC078B3F98F08B3FD8
:104CA00019F4809175040EC08C3F19F4809177043B
:104CB00009C08D3F19F48091790404C08E3F21F41E
:104CC00080917B048093A9038091CD078B3F98F05E
:104CD0008B3F19F4809175040EC08C3F19F48091BC
:104CE000770409C08D3F19F48091790404C08E3F88
:104CF00021F480917B04809395048091CE078B3FB3
:104D000098F08B3F19F4809175040EC08C3F19F414
:104D10008091770409C08D3F19F48091790404C013
:104D20008E3F21F480917B04809396048091CF077D
:104D30008B3F98F08B3F19F4809175040EC08C3F27
:104D400019F48091770409C08D3F19F4809179049A
:104D500004C08E3F21F480917B048093970480915E
:104D6000D0078B3F98F08B3F19F4809175040EC0EB
:104D70008C3F19F48091770409C08D3F19F480911C
:104D8000790404C08E3F21F480917B0480939804C1
:104D90008091E0078B3F98F08B3F19F48091750468
:104DA0000EC08C3F19F48091770409C08D3F19F42F
:104DB0008091790404C08E3F21F480917B0480931C
:104DC00099048091E1078B3F98F08B3F19F4809113
:104DD00075040EC08C3F19F48091770409C08D3F93
:104DE00019F48091790404C08E3F21F480917B04F2
:104DF00080939A048091E2078B3F98F08B3F19F4DF
:104E0000809175040EC08C3F19F48091770409C01D
:104E10008D3F19F48091790404C08E3F21F4809174
:104E20007B0480939B048091E3078B3F98F08B3F3A
:104E300019F4809175040EC08C3F19F480917704A9
:104E400009C08D3F19F48091790404C08E3F21F48C
:104E500080917B0480939C048091D1078B3F98F0D4
:104E60008B3F19F4809175040EC08C3F19F480912A
:104E7000770409C08D3F19F48091790404C08E3FF6
:104E800021F480917B048093AA038091D6078B3F05
:104E900098F08B3F19F4809175040EC08C3F19F483
:104EA0008091770409C08D3F19F48091790404C082
:104EB0008E3F21F480917B048093AB038091D907CE
:104EC0008B3F98F08B3F19F4809175040EC08C3F96
:104ED00019F48091770409C08D3F19F48091790409
:104EE00004C08E3F21F480917B0480939D048091C7
:104EF000DA078B3F98F08B3F19F4809175040EC050
:104F00008C3F19F48091770409C08D3F19F480918A
:104F1000790404C08E3F21F480917B0480939E0429
:104F20008091DF078B3F98F08B3F19F480917504D7
:104F30000EC08C3F19F48091770409C08D3F19F49D
:104F40008091790404C08E3F21F480917B0480938A
:104F5000AC038091E5078B3F98F08B3F19F480916B
:104F600075040EC08C3F19F48091770409C08D3F01
:104F700019F48091790404C08E3F21F480917B0460
:104F80008093340880913408823010F481E002C0AC
:104F90008F3F11F4809334088091E7078B3F98F09E
:104FA0008B3F19F4809175040EC08C3F19F48091E9
:104FB000770409C08D3F19F48091790404C08E3FB5
:104FC00021F480917B0480935908809159088230A4
:104FD00010F481E002C08F3F11F480935908809152
:104FE000E8078B3F98F08B3F19F4809175040EC051
:104FF0008C3F19F48091770409C08D3F19F480919A
:10500000790404C08E3F21F480917B0480931308BF
:105010008091E9078B3F98F08B3F19F480917504DC
:105020000EC08C3F19F48091770409C08D3F19F4AC
:105030008091790404C08E3F21F480917B04809399
:105040006B088091EA078B3F98F08B3F19F48091B1
:1050500075040EC08C3F19F48091770409C08D3F10
:1050600019F48091790404C08E3F21F480917B046F
:1050700080930C088091EB078B3F98F08B3F19F4DD
:10508000809175040EC08C3F19F48091770409C09B
:105090008D3F19F48091790404C08E3F21F48091F2
:1050A0007B04809319088091EC078B3F98F08B3F2D
:1050B00019F4809175040EC08C3F19F48091770427
:1050C00009C08D3F19F48091790404C08E3F21F40A
:1050D00080917B04809375088091EF078B3F98F057
:1050E0008B3F19F4809175040EC08C3F19F48091A8
:1050F000770409C08D3F19F48091790404C08E3F74
:1051000021F480917B0480936C088091ED078B3FA4
:1051100098F08B3F19F4809175040EC08C3F19F400
:105120008091770409C08D3F19F48091790404C0FF
:105130008E3F21F480917B0480931F088091F407B7
:105140008B3F98F08B3F19F4809175040EC08C3F13
:1051500019F48091770409C08D3F19F48091790486
:1051600004C08E3F21F480917B048093730860918A
:10517000A90370E080E090E00E94375627E137EB0A
:1051800041ED58E30E94ED5660939D0370939E039A
:1051900080939F039093A0038091C30780935A0844
:1051A0008091C20780931A0808951F93CF93DF93CD
:1051B000182FC4E6D0E00DC01150809186048823DA
:1051C00051F4D093DA03C093D9038AEF90E00E94A0
:1051D0000411112389F7DF91CF911F9108958091D8
:1051E0008604882321F51092140810920B0810925F
:1051F0003F0810924C088091C803882311F08093D7
:105200000B088091C903882311F0809314088091C2
:10521000CA03882311F080934C088091CB03882324
:1052200011F080933F088091AB048C7F03C0809184
:10523000AB0481608093AB0480910B08EAE3F7E054
:1052400080933A0710923B078091140880933C07A3
:10525000138280914C0880933E07158280913F080D
:1052600080934007178210920D0410920E040E9442
:10527000061D0895809100018D3011F40E944A1599
:1052800010927A008091E6039091E70390931608BC
:10529000809315088091E8039091E90390930A08A0
:1052A000809309088091EA039091EB0390935C0846
:1052B00080935B086091EE037091EF03882777FD80
:1052C0008095982F2CE030E040E050E00E9450574D
:1052D00070935108609350086091EC037091ED0356
:1052E000882777FD8095982F0E94505770936A0801
:1052F000609369088091F0039091F10390932508E1
:10530000809324088FEE80937A008091B407E82F71
:10531000F0E0EE0FFF1FE258F84F8081918120915D
:1053200075043091760483599F4F821793071CF0C0
:105330002F5F3F4F0CC08081918182599F4F821710
:1053400093074CF42115310531F021503040309352
:105350007604209375048091B507E82FF0E0EE0FF6
:10536000FF1FE258F84F808191812091770430919E
:10537000780483599F4F821793071CF02F5F3F4F8C
:105380000CC08081918182599F4F821793074CF402
:105390002115310531F021503040309378042093AD
:1053A00077048091B607E82FF0E0EE0FFF1FE25878
:1053B000F84F808191812091790430917A0483594A
:1053C0009F4F821793071CF02F5F3F4F0CC08081C7
:1053D000918182599F4F821793074CF42115310513
:1053E00031F02150304030937A0420937904809139
:1053F000B707E82FF0E0EE0FFF1FE258F84F80816B
:10540000918120917B0430917C0483599F4F8217B6
:1054100093071CF02F5F3F4F0CC080819181825910
:105420009F4F821793074CF42115310531F021501D
:10543000304030937C0420937B04809175049091DC
:10544000760497FF05C010927604109275040AC086
:105450008F3F910539F034F08FEF90E09093760410
:1054600080937504809177049091780497FF05C02C
:1054700010927804109277040AC08F3F910539F09A
:1054800034F08FEF90E090937804809377048091CC
:10549000790490917A0497FF05C010927A041092D3
:1054A00079040AC08F3F910539F034F08FEF90E016
:1054B00090937A048093790480917B0490917C048A
:1054C00097FF05C010927C0410927B040AC08F3FA6
:1054D000910539F034F08FEF90E090937C04809345
:1054E0007B046091DB0770E080E090E024EC39E021
:1054F00040E050E00E9450576093950370939603EC
:1055000080939703909398036091DC0770E080E0AC
:1055100090E00E9450576093990370939A03809390
:105520009B0390939C030895469A10921F04109237
:105530001E04109221041092200480E090E0A0E06C
:10554000B0E08093240490932504A0932604B093A4
:10555000270410921504109214041092170410924C
:105560001604109219041092180410923A0810921E
:10557000390810929D0410929E041092F8030E9424
:105580003A2984E690E00E941A110E943A298091FB
:10559000B80780FF10C08091170390911803875BB4
:1055A000934038F480911703909118038E5E9240D7
:1055B00010F40E9409164091E6035091E7035093BE
:1055C0001504409314042091E8033091E9033093CB
:1055D0001704209316048091EA039091EB039093B3
:1055E0001904809318048091EA039091EB0390933F
:1055F0003A088093390830931B0420931A0450937F
:105600001D0440931C04F999FECF24E030E032BD24
:1056100021BDF89A80B5853038F180916908909164
:105620006A0897FF03C0909581959F4F6CE070E0EA
:105630000E948F577093210460932004809150083A
:105640009091510897FF03C0909581959F4F6CE012
:1056500070E00E948F5770931F0460931E04609146
:1056600066077091670742C0F999FECF32BD21BD30
:10567000F89A30B5F999FECF85E090E092BD81BDF2
:10568000F89A20B5932F80E0820F911D90931F040C
:1056900080931E04F999FECF86E090E092BD81BD13
:1056A000F89A30B5F999FECF87E090E092BD81BDC0
:1056B000F89A20B5932F80E0820F911D90932104DA
:1056C00080932004F999FECF88E090E092BD81BDDF
:1056D000F89A30B5F999FECF89E090E092BD81BD8E
:1056E000F89A20B5732F60E0620F711D882777FD4F
:1056F0008095982F0E943956609324047093250456
:10570000809326049093270410924A0410924B042D
:1057100010924C0410924D0410924E0410924F04BB
:10572000109250041092510410925204109253049B
:10573000109254041092550410925604109257047B
:10574000109258041092590410925A0410925B045B
:1057500010925C0410925D041092160810921508C5
:1057600010920A081092090810925C0810925B08C7
:1057700084E690E00E941A11809113039091140323
:10578000A0911503B0911603909369078093680761
:105790001092FA031092F9031092620410926304BB
:1057A00010926404109265048091660490916704DD
:1057B00090936904809368040E94804782E390E09C
:1057C0009093DA038093D9036091DB0770E080E067
:1057D00090E024EC39E040E050E00E9450576856D9
:1057E000754C8F4F9F4F60939503709396038093F2
:1057F0009703909398036091DC0770E080E090E05D
:105800000E9450576856754C8F4F9F4F6093990375
:1058100070939A0380939B0390939C031092AE0322
:105820001092AD036091660470916704882777FD3C
:105830008095982F2BE035E040E050E00E945057D3
:105840006093650870936608809367089093680872
:105850001092700410926F0481E0809301010E9405
:1058600070548091AB0484608093AB048FEF80937D
:1058700065098091DE0790E024E0880F991F2A9542
:10588000E1F78093660980E280936709609166047E
:1058900070916704882777FD8095982F2BE035E07D
:1058A00040E050E00E94505760936F08709370087A
:1058B000809371089093720808952F923F924F92AF
:1058C0005F926F927F928F929F92AF92BF92CF9290
:1058D000DF92EF92FF920F931F93DF93CF93CDB799
:1058E000DEB762970FB6F894DEBF0FBECDBF0E9441
:1058F000FE1E8091DD089091DE08009729F0019747
:105900009093DE088093DD080E945848892B49F463
:10591000809100018A3011F0843111F4289A01C07D
:105920002898809100018C3010F4299A01C02998A0
:1059300020918404309185043A83298380911A0848
:10594000282F30E0C901099649815A8184179507AB
:1059500024F0C9010A969A83898380917D04843654
:1059600008F06EC080910501882399F480910B03A3
:1059700090910C038F5F9F4F61F488E99AE39093B5
:10598000DA038093D90380E09CE090930C0380932A
:105990000B038091CD049091CE04009731F00197D4
:1059A0009093CE048093CD0404C01092860410928C
:1059B0006C04809100018A3011F0843111F4289A2E
:1059C00001C028988091A9049091AA04895E93400F
:1059D000A0F18091C907E82FF0E0FA83E98381E024
:1059E00080936C04A091B007B0E0AA0FBB1FFD012B
:1059F000EC56F84F11821082E091B1072E2F30E063
:105A0000220F331FC9018C56984FFC01118210825E
:105A1000A258B84F11961C921E922258384FD901A5
:105A200011961C921E92E091B307F0E0EE0FFF1F5B
:105A3000E258F84F11821082F6C210928604F3C227
:105A400080917D048D3808F4EEC210926C04809130
:105A5000CA0722E3829FC00111249093CE04809351
:105A6000CD04E981FA81B9978CF08091860488236E
:105A700069F08091A9049091AA04FFEF8F3F9F07DE
:105A800029F001969093AA048093A9048091A90417
:105A90009091AA048F3F910509F038F51092E70420
:105AA0001092E8041092E9041092EA041092E304C0
:105AB0001092E4041092E5041092E6048A3F9105E6
:105AC000C9F481E08093C6041092DF041092E004D0
:105AD0001092E1041092E20410925A0410925B04B6
:105AE00010925C0410925D0405C08091AB0482604A
:105AF0008093AB04E091B207F0E0EE0FFF1FE25895
:105B0000F84F80819181813591050CF4D9C1809144
:105B10008604882309F0D4C18091B307E82FF0E010
:105B2000EE0FFF1FE258F84F808191818C34910570
:105B30000CF406C18091CC048F5F8093CC04893C27
:105B400008F4BEC1809100018C3010F4299801C086
:105B5000299A0E94942A109286041092CC041092E2
:105B6000AA041092A9048091B007482F50E0FA01CE
:105B7000EE0FFF1FE258F84F808191818734910525
:105B80009CF4E091B107F0E0EE0FFF1FE258F84FF0
:105B90000190F081E02DF7FF03C0F095E195FF4FF4
:105BA000E734F1050CF46EC08091B107A82FB0E086
:105BB000FD01EE0FFF1FE258F84F8081918187347D
:105BC000910544F0FA01EE0FFF1FE258F84F0190E3
:105BD000F081E02DFD01EE0FFF1FE258F84F8081AC
:105BE00091818734910564F0FA01EE0FFF1FE258AE
:105BF000F84F808191818734910514F022E001C033
:105C000021E0FD01EE0FFF1FE258F84F80819181E6
:105C1000863491055CF4FA01EE0FFF1FE258F84F4D
:105C200080819181873491050CF023E0FD01EE0F16
:105C3000FF1FE258F84F808191818A5B9F4F5CF48F
:105C4000FA01EE0FFF1FE258F84F808191818734EF
:105C500091050CF024E0AA0FBB1FA258B84F8D91FC
:105C60009C918A5B9F4F5CF4440F551F4258584FDC
:105C7000FA0180819181863491050CF425E0822F10
:105C80000E943E03E091B107F0E0EE0FFF1FE258E3
:105C9000F84F0190F081E02DF7FF03C0F095E195FA
:105CA000FF4F7E97B4F4E091B007F0E0EE0FFF1FD6
:105CB000E258F84F808191818A5B9F4F54F481E0D4
:105CC00080937B0688EE93E09093DA038093D90368
:105CD000F7C00E94230346E560EB77E00E94B7031C
:105CE0008091B80780FF10C080911703909118032E
:105CF000875B934038F480911703909118038E5E70
:105D0000924010F40E9409160E94942A0E942303D4
:105D10000E94D5280E94AD488091C708882309F4C5
:105D2000CFC088EE93E00E94041188EE93E0909338
:105D3000DA038093D90384EF91E00E940411C0C07C
:105D400080819181855B9F4F0CF0B8C08091CC041D
:105D50008F5F8093CC04893C08F4B2C0809100012D
:105D60008C3010F4299801C0299AF999FECF1FBAF6
:105D700004E010E012BD01BD8FEF80BD0FB6F894B6
:105D8000FA9AF99A0FBE109286041092CC041092DF
:105D9000AA041092A9040E94942A20911E04309112
:105DA0001F04F999FECF1FBA12BD01BDC90160E001
:105DB00071E00E948F5760BD0FB6F894FA9AF99A75
:105DC0000FBEF999FECF1FBA85E090E092BD81BD6C
:105DD000C90160E071E00E948F5780BD0FB6F89452
:105DE000FA9AF99A0FBE2091200430912104F99972
:105DF000FECF1FBA86E090E092BD81BDC90160E090
:105E000071E00E948F5760BD0FB6F894FA9AF99A24
:105E10000FBEF999FECF1FBA87E090E092BD81BD19
:105E2000C90160E071E00E948F5780BD0FB6F89401
:105E3000FA9AF99A0FBE20912404309125044091DA
:105E4000260450912704F999FECF1FBA88E090E00C
:105E500092BD81BDCA01B9010E940656DC01CB0189
:105E600060E071E00E948F5760BD0FB6F894FA9A17
:105E7000F99A0FBE20912404309125044091260404
:105E800050912704F999FECF1FBA89E090E092BDA6
:105E900081BDCA01B9010E940656DC01CB0160E058
:105EA00071E00E948F5780BD0FB6F894FA9AF99A64
:105EB0000FBE0E9423030E94D52802C01092CC047A
:105EC000E091B207F0E0EE0FFF1FE258F84F80813B
:105ED00091818B5A9F4F0CF0A6C0E091B307F0E080
:105EE000EE0FFF1FE258F84F80819181855B9F4F35
:105EF0000CF077C08091CB048F5F8093CB04893CFA
:105F000008F471C0469A88EC8093CB0481E090E05D
:105F10009093AA048093A90481E080938604109250
:105F2000DF041092E0041092E1041092E204109257
:105F30005A0410925B0410925C0410925D0410925B
:105F40005E0410925F04109260041092610410923B
:105F50004A0410924B0410924C0410924D0410927B
:105F600052041092530410925404109255048091DC
:105F70002A0490912B04A0912C04B0912D048093BD
:105F80004E0490934F04A0935004B0935104809119
:105F9000320490913304A0913404B091350480937D
:105FA000560490935704A0935804B0935904109248
:105FB000E7041092E8041092E9041092EA041092A7
:105FC000E3041092E4041092E5041092E60480E0E9
:105FD00090E00E94024A8091AB0488608093AB04F9
:105FE00002C01092CB04E091B307F0E0EE0FFF1F68
:105FF000E258F84F808191818C34910594F0809122
:10600000CA048F5F8093CA04893C68F04698109256
:10601000860488EC8093CA041092AA041092A90402
:1060200002C01092CA048091770381508093770355
:106030008F5F29F080916C04882309F4F0C20E94DC
:106040007A258091B007082F10E0000F111FF8018A
:10605000E258F84F208131818091BF07A82EBB24E0
:106060002A9DC0012B9D900D3A9D900D11244091C9
:10607000BC045091BD049A01220F331F240F351F19
:10608000820F931F64E070E00E948F577093BD04ED
:106090006093BC040C56184FF801808191810091E7
:1060A000C00710E0AC01409FC001419F900D509F80
:1060B000900D1124860F971F9093BD048093BC040C
:1060C0002091F7043091F8044091F3045091F404C6
:1060D0006C01C21AD30AC41AD50AD0927F04C092A6
:1060E0007E048091B107E82EFF24EE0CFF1CF7011F
:1060F000E258F84F80819181DC01AA9DC001AB9DDF
:10610000900DBA9D900D11244091BA045091BB049A
:106110009A01220F331F240F351F820F931F64E053
:1061200070E00E948F577093BB046093BA04E4E957
:10613000F7E0EE0EFF1ED7018D919C91FC01E09FD0
:10614000C001E19F900DF09F900D1124860F971FC5
:106150009093BB048093BA042091F9043091FA041F
:106160004091F5045091F6044C01821A930A841A66
:10617000950A9092810480928004E091B307F0E048
:10618000EE0FFF1FE258F84F808191810027112701
:10619000081B190B1093830400938204E091B2074B
:1061A000F0E0EE0FFF1FE258F84FE080F18028E7A3
:1061B00030E0E20EF31EF0928504E09284046091D8
:1061C000A60370E080E090E00E94375620E030E0C7
:1061D00040E251E40E94365520E030E040E85CE3C4
:1061E0000E94ED5660936008709361088093620886
:1061F000909363086091A70370E080E090E00E94B4
:10620000375620E030EE4BE256E40E949E556093F4
:106210003B0870933C0880933D0890933E08809122
:10622000870680FF54C080917308813808F44FC0FE
:1062300080918006992787FD9095AC01A49EC001AE
:10624000A59E900DB49E900D1124C80ED91ED0921B
:106250007F04C0927E0480918106992787FD9095E6
:10626000DC01AA9EC001AB9E900DBA9E900D112438
:10627000880E991E909281048092800480918206FB
:10628000992787FD9095080F191F10938304009399
:1062900082042091BD0730E080918406992787FD14
:1062A0009095FC012E9FC0012F9F900D3E9F900D59
:1062B00011249093AE038093AD038091830690E008
:1062C0008E159F0524F49093850480938404809117
:1062D00084049091850497FF04C010928504109265
:1062E00084048091B80782FF0CC080E090E0A0E0B9
:1062F000B0E080933B0890933C08A0933D08B09396
:106300003E0820E030E040E050E06091600870918D
:10631000610880916208909163080E949A558823D1
:1063200064F480E090E0A0E0B0E080936008909397
:106330006108A0936208B093630820E030E040E079
:1063400050E060913B0870913C0880913D0890912D
:106350003E080E949A55882364F480E090E0A0E013
:10636000B0E080933B0890933C08A0933D08B09325
:106370003E0840917E0410917F04E091A504F091C5
:10638000A604842F912F64E070E00E948F57CB0108
:1063900077FF03C0909581959F4FE817F907DCF4CC
:1063A000842F912F9C0137FF03C0309521953F4FDB
:1063B000C90195958795959587959093A6048093A7
:1063C000A5048536910564F084E690E09093A604D8
:1063D0008093A50405C03197F093A604E093A5042B
:1063E0004091800410918104E091A704F091A804E9
:1063F000842F912F64E070E00E948F57CB0177FFCC
:1064000003C0909581959F4FE817F907DCF4842F1E
:10641000912F9C0137FF03C0309521953F4FC90153
:1064200095958795959587959093A8048093A70453
:106430008536910564F084E690E09093A8048093FB
:10644000A70405C03197F093A804E093A7048091B6
:106450006C04882341F01092A6041092A5041092B7
:10646000A8041092A7048091B107A82FB0E0FD0105
:10647000EE0FFF1FE258F84F208131818091D7073E
:10648000482F50E04217530744F48091F50782FFEC
:1064900004C081E0809391040FC0AA0FBB1FA258D3
:1064A000B84F2D913C918091D807481B5109241772
:1064B000350714F4109291048091B107A82FB0E031
:1064C000FD01EE0FFF1FE258F84F208131818091CE
:1064D000D707482F50E088279927841B950B28174A
:1064E000390744F48091F50783FF04C081E080936D
:1064F000920414C080919204882381F0AA0FBB1FDC
:10650000A258B84F2D913C918091D80790E0841B00
:10651000950B8217930714F4109292048091B007A0
:10652000A82FB0E0FD01EE0FFF1FE258F84F2081C9
:1065300031818091D707482F50E04217530744F428
:106540008091F50780FF04C081E08093940413C01C
:1065500080919404882379F0AA0FBB1FA258B84FEA
:106560002D913C918091D807481B5109241735077C
:1065700014F4109294048091B007A82FB0E0FD01AC
:10658000EE0FFF1FE258F84F208131818091D7072D
:10659000482F50E088279927841B950B2817390727
:1065A00044F48091F50781FF04C081E08093930457
:1065B00014C080919304882381F0AA0FBB1FA258B6
:1065C000B84F2D913C918091D80790E0841B950B9A
:1065D0008217930714F410929304809191048823F6
:1065E00021F480919204882321F081E0809390042B
:1065F00002C01092900480919404882321F4809129
:106600009304882351F081E080938F0410929004CA
:10661000109291041092920402C010928F04809103
:106620009004882321F480918F04882351F0809175
:10663000D60790E029813A818217930714F49A8350
:10664000898380916C04882341F110928304109215
:10665000820410927F0410927E04109281041092A2
:10666000800480E090E0A8ECBFE380936008909302
:106670006108A0936208B09363088BE09CEBA2E3EF
:10668000BCE380933B0890933C08A0933D08B093F3
:106690003E081092900410928F0480912E089091E1
:1066A0002F08A0913008B091310820912A04309130
:1066B0002B0440912C0450912D04820F931FA41F92
:1066C000B51F80932E0890932F08A0933008B093A5
:1066D00031088091350890913608A0913708B09123
:1066E00038082091320430913304409134045091A1
:1066F0003504820F931FA41FB51F80933508909314
:106700003608A0933708B0933808809120089091FC
:106710002108A0912208B091230820912E043091E5
:106720002F044091300450913104820F931FA41F15
:10673000B51F8093200890932108A0932208B0935E
:10674000230880910F0890911008A0911108B09132
:10675000120820913604309137044091380450914A
:106760003904820F931FA41FB51F80930F089093C5
:106770001008A0931108B093120880918F04882309
:1067800029F480919004882309F45CC010923A04A3
:1067900010923B0410923C0410923D0410923E046F
:1067A00010923F04109240041092410410922E085F
:1067B00010922F081092300810923108109235086C
:1067C000109236081092370810923808109220085C
:1067D00010922108109222081092230810920F089C
:1067E00010921008109211081092120880914A0419
:1067F00090914B04A0914C04B0914D0480934E04B1
:1068000090934F04A0935004B0935104809152048C
:1068100090915304A0915404B09155048093560470
:1068200090935704A0935804B09359041092FC031A
:106830001092FB0310928E0410928D0410928C041F
:1068400010928B0480918F04882309F000C28091FC
:106850009004882309F0FBC12091650960912A0406
:1068600070912B0480912C0490912D04609032043F
:106870007090330480903404909035044091A504C6
:106880005091A604588B4F872090500830905108A3
:106890004090690850906A082F3F09F4DCC0E090EE
:1068A000C407FF2400E010E0A22EBB24A7FCB09494
:1068B000CB2CDB2CA80197010E94C457C101AA2749
:1068C00097FDA095BA2F281B390B4A0B5B0BCA0109
:1068D000B901A60195010E94505720E032E040E046
:1068E00050E00E94C4572B873C874D875E872F83DB
:1068F000388749875A87C401B301A80197010E94CC
:10690000C457C201AA2797FDA095BA2F281B390B9F
:106910004A0B5B0BCA01B901A60195010E945057B1
:1069200020E032E040E050E00E94C457122F032FD5
:10693000F42EE52E222E332E442E552E8F85988947
:10694000813491053CF48091A7049091A80481348E
:106950009105D4F06B857C858D859E8522E030E0A5
:1069600040E050E00E94C4572F83388749875A87F8
:10697000612F702F8F2D9E2D22E030E040E050E0FF
:106980000E94C45719012A01E091B307F0E0EE0F0D
:10699000FF1FE258F84F0190F081E02DF7FF03C090
:1069A000F095E195FF4F7A97C4F06F8178858985DE
:1069B0009A8523E030E040E050E00E94C4572F83E6
:1069C000388749875A87B101C20123E030E040E0AF
:1069D00050E00E94C45719012A0160916709662E90
:1069E000772467FC7094872C972C2F8138854985F4
:1069F0005A85C901DA019C01AD016216730684064D
:106A0000950614F4A4019301862F992787FD90958C
:106A1000909581959F4F7C010027F7FC0095102FE2
:106A200059016A012E153F054007510714F457011B
:106A30006801C101D201681679068A069B0614F422
:106A4000D401C3018E159F05A007B1070CF4D7C070
:106A50007C018D01D4C0E090C407FF2400E010E069
:106A6000A80197010E94C45759016A01C101AA27D0
:106A700097FDA095BA2FA81AB90ACA0ADB0AC40161
:106A8000B301A80197010E94C45779018A01C2018C
:106A9000AA2797FDA095BA2FE81AF90A0A0B1B0B33
:106AA000C601B50120E130E040E050E00E94C4574B
:106AB000922E832E742E652E822F932FA42FB52F06
:106AC0005C016D01C801B70120E130E040E050E019
:106AD0000E94C457222E532E442E352E822F932FE0
:106AE000A42FB52F7C018D01AF85B889A134B105E4
:106AF0003CF48091A7049091A80481349105E4F0BE
:106B0000692D782D872D962D23E030E040E050E070
:106B10000E94C457C901DA015C016D01622D752D17
:106B2000842D932D23E030E040E050E00E94C457D4
:106B3000C901DA017C018D01E091B307F0E0EE0FAD
:106B4000FF1FE258F84F0190F081E02DF7FF03C0DE
:106B5000F095E195FF4F7A97C4F0C601B50123E0A7
:106B600030E040E050E00E94C457C901DA015C0106
:106B70006D01C801B70123E030E040E050E00E9421
:106B8000C457C901DA017C018D01B1E2AB16B10431
:106B9000C104D10434F040E2A42EB12CC12CD12C7C
:106BA00011C0E0EEAE16EFEFBE06EFEFCE06EFEF50
:106BB000DE0644F430EEA32E3FEFB32E3FEFC32E9C
:106BC0003FEFD32EF1E2EF16F1040105110534F089
:106BD00020E2E22EF12C012D112D11C020EEE21643
:106BE0002FEFF2062FEF02072FEF120744F490EE7B
:106BF000E92E9FEFF92E9FEF092F9FEF192F80911C
:106C00004A0490914B04A0914C04B0914D048A1910
:106C10009B09AC09BD0980934A0490934B04A0934F
:106C20004C04B0934D048091520490915304A09170
:106C30005404B09155048E199F09A00BB10B809399
:106C4000520490935304A0935404B093550480913C
:106C5000FB039091FC038F3F910509F008F46EC58A
:106C600080918F04882309F0EBC4809190048823DD
:106C700009F0E6C480916E04882309F0E1C46091B4
:106C80002E0870912F08809130089091310820E0F3
:106C900031E040E050E00E94C45759016A0120935E
:106CA0002E0830932F08409330085093310860919C
:106CB000350870913608809137089091380820E0A7
:106CC00031E040E050E00E94C45739014A0120936E
:106CD0003508309336084093370850933808E090D1
:106CE000C407FF2400E010E020913A0430913B04F7
:106CF00040913C0450913D04C801B7010E94505797
:106D000020E031E040E050E00E94C4572B833C83F8
:106D10004D835E8320933A0430933B0440933C04BC
:106D200050933D0420913E0430913F044091400433
:106D300050914104C801B7010E94505720E031E052
:106D400040E050E00E94C45719012A0120933E04FC
:106D500030933F04409340045093410460914204B7
:106D600070914304809144049091450420E031E007
:106D700040E050E00E94C457209342043093430403
:106D800040934404509345048B819C81AD81BE8126
:106D9000A81AB90ACA0ADB0AA092D304B092D40492
:106DA000C092D504D092D604E090DD07FF2400E025
:106DB00010E0C601B501A80197010E94C45759010E
:106DC0006A012093C2043093C3044093C4045093D7
:106DD000C50462187308840895086092CF04709205
:106DE000D0048092D1049092D204C401B301A801CE
:106DF00097010E94C45779018A012093BE04309301
:106E0000BF044093C0045093C104C601B50120E003
:106E100031E040E050E00E94C45730938E0420934C
:106E20008D04C801B70120E031E040E050E00E944D
:106E3000C45730938C0420938B048091A5049091C7
:106E4000A60481349105C4F48091A7049091A8040C
:106E5000813491058CF4E091B307F0E0EE0FFF1F51
:106E6000E258F84F0190F081E02DF7FF03C0F09554
:106E7000E195FF4F7A97E4F0809165098F3FC1F467
:106E800080918D0490918E0462E070E00E948F5793
:106E900070938E0460938D0480918B0490918C0488
:106EA00062E070E00E948F5770938C0460938B04B3
:106EB0006091200870912108809122089091230808
:106EC00020E031E040E050E00E94C45720932008C9
:106ED00030932108409322085093230860910F08B3
:106EE00070911008809111089091120820E031E013
:106EF00040E050E00E94C45720930F0830931008E0
:106F00004093110850931208E0902E04F0902F0443
:106F1000009130041091310480912A0490912B0447
:106F2000A0912C04B0912D04E81AF90A0A0B1B0B4E
:106F3000E092DB04F092DC040093DD041093DE04A5
:106F4000209136043091370440913804509139042F
:106F50008091320490913304A0913404B0913504AF
:106F6000281B390B4A0B5B0B2093D7043093D804B2
:106F70004093D9045093DA04E092D304F092D404FD
:106F80000093D5041093D6042093CF043093D004FB
:106F90004093D1045093D20480914E0490914F04B9
:106FA000A0915004B09151048E199F09A00BB10B10
:106FB00080934E0490934F04A0935004B0935104D7
:106FC0008091560490915704A0915804B0915904AF
:106FD000821B930BA40BB50B80935604909357041C
:106FE000A0935804B09359041092700410926F0447
:106FF00080916F0890917008A0917108B09172080B
:107000008837E7E19E07E7E0AE07E0E0BE0764F0FF
:1070100088579741A740B04080936F0890937008BD
:10702000A0937108B093720880916F0890917008D6
:10703000A0917108B0917208B7FF0CC08858984EA3
:10704000A84FBF4F80936F0890937008A09371086A
:10705000B0937208809100018A3011F0843111F4EC
:10706000289801C0289A81E090E09093B904809319
:10707000B8048091B0049091B104A091B204B09191
:10708000B30420912E0830912F0840913008509180
:107090003108821B930BA40BB50B815E914BAF4F54
:1070A000BF4F8F539C49A040B04028F080916609A3
:1070B00081330CF4D7C02091D3043091D404409193
:1070C000D5045091D604213080E1380780E048078C
:1070D00080E058070CF453C08091B704882309F46A
:1070E0004AC0DA01C9010CE0B595A7959795879537
:1070F0000A95D1F701969093B9048093B804CA0118
:10710000B90128E030E040E050E00E94C457C901D6
:10711000DA018093C2049093C304A093C404B09393
:10712000C50489589341A040B04064F088E893E1D9
:10713000A0E0B0E08093C2049093C304A093C40481
:10714000B093C5046091C2047091C3048091C404DB
:107150009091C50420E031E040E050E00E94C45727
:1071600080918D0490918E04820F931F90938E04D2
:1071700080938D0406C081E08093B70402C0109212
:10718000B7044091D3045091D4046091D504709118
:10719000D6044030F0EF5F07FFEF6F07FFEF7F0788
:1071A0000CF05DC08091B604882309F454C0882790
:1071B0009927DC01841B950BA60BB70B1CE0B5953A
:1071C000A795979587951A95D1F72091B804309196
:1071D000B904280F391F3093B9042093B804CB01A8
:1071E000BA0128E030E040E050E00E94C457C901F5
:1071F000DA018093C2049093C304A093C404B093B3
:10720000C50488579C4EAF4FBF4F64F488E79CEE8F
:10721000AFEFBFEF8093C2049093C304A093C40464
:10722000B093C5046091C2047091C3048091C404FA
:107230009091C50420E031E040E050E00E94C45746
:1072400080918D0490918E04820F931F90938E04F1
:1072500080938D0411C081E08093B6040DC010921C
:10726000B6040AC01092B9041092B80488EE93E0F4
:1072700090939403809393038091DE07282F30E04E
:107280008091B8049091B9042817390724F43093F9
:10729000B9042093B804409166098091B804909194
:1072A000B904A4E0880F991FAA95E1F7242F33278A
:1072B00027FD3095281739077CF4242F47FD215FDF
:1072C0002595259525952595822F992787FD9095BC
:1072D0009093B9048093B8048091D3049091D4041E
:1072E000A091D504B091D60481509440A040B04004
:1072F00074F080911404909115042091B804309199
:10730000B904820F931F9093150480931404809105
:10731000D3049091D404A091D504B091D6048050A8
:107320009C4FAF4FBF4F74F480911404909115049B
:107330002091B8043091B904821B930B90931504EB
:107340008093140481E090E09093B9048093B80492
:107350001092BE041092BF041092C0041092C10497
:107360008091AC049091AD04A091AE04B091AF04B3
:1073700020913508309136084091370850913808EF
:10738000821B930BA40BB50B815E914BAF4FBF4F8C
:107390008F539C49A040B04028F08091660981330A
:1073A0000CF4DDC0E090CF04F090D0040091D10443
:1073B0001091D20481E0E81680E1F80680E0080729
:1073C00080E018070CF458C08091B504882309F4B4
:1073D0004FC0A8019701FCE0559547953795279533
:1073E000FA95D1F78091B8049091B904820F931F58
:1073F0009093B9048093B804C801B70128E030E045
:1074000040E050E00E94C457C901DA018093BE04F5
:107410009093BF04A093C004B093C10489589341D2
:10742000A040B04064F088E893E1A0E0B0E0809331
:10743000BE049093BF04A093C004B093C1046091B4
:10744000BE047091BF048091C0049091C10420E0FB
:1074500031E040E050E00E94C45780918B0490914D
:107460008C04820F931F90938C0480938B0406C02E
:1074700081E08093B50402C01092B5044091CF041E
:107480005091D0046091D1047091D2044030F0EF5B
:107490005F07FFEF6F07FFEF7F070CF05DC0809184
:1074A000B404882309F454C088279927DC01841B7D
:1074B000950BA60BB70BECE0B595A795979587951F
:1074C000EA95D1F72091B8043091B904280F391FFB
:1074D0003093B9042093B804CB01BA0128E030E01E
:1074E00040E050E00E94C457C901DA018093BE0415
:1074F0009093BF04A093C004B093C10488579C4EDE
:10750000AF4FBF4F64F488E79CEEAFEFBFEF8093BF
:10751000BE049093BF04A093C004B093C1046091D3
:10752000BE047091BF048091C0049091C10420E01A
:1075300031E040E050E00E94C45780918B0490916C
:107540008C04820F931F90938C0480938B0411C042
:1075500081E08093B4040DC01092B4040AC010926C
:10756000B9041092B80488EE93E09093940380934A
:1075700093038091DE07282F30E08091B80490912A
:10758000B9042817390724F43093B9042093B804B8
:10759000409166098091B8049091B90454E0880F35
:1075A000991F5A95E1F7242F332727FD3095281787
:1075B00039077CF4242F47FD215F259525952595D6
:1075C0002595822F992787FD90959093B9048093F4
:1075D000B8048091CF049091D004A091D104B091CF
:1075E000D20481509440A040B04074F080911604C1
:1075F000909117042091B8043091B904820F931F21
:1076000090931704809316048091CF049091D00436
:10761000A091D104B091D20480509C4FAF4FBF4F86
:10762000CCF480911604909117042091B804309105
:10763000B904821B930B90931704809316040AC01D
:1076400010928C0410928B0410928E0410928D0470
:1076500010926E0420E030E040E050E060913B0882
:1076600070913C0880913D0890913E080E949A5587
:10767000882341F410928C0410928B0410928E0493
:1076800010928D0480912E0890912F08A0913008BF
:10769000B09131088093B0049093B104A093B204E8
:1076A000B093B3048091350890913608A0913708C3
:1076B000B09138088093AC049093AD04A093AE04CD
:1076C000B093AF0410923A0410923B0410923C0421
:1076D00010923D0410923E0410923F041092400418
:1076E00010924104109242041092430410924404F8
:1076F0001092450410922E0810922F081092300814
:1077000010923108109235081092360810923708FE
:107710001092380810922008109221081092220826
:107720001092230810920F0810921008109211085E
:10773000109212081092FC031092FB038091DE035A
:10774000882309F467C28091E1039091E203892BB9
:1077500009F460C21092DE03209150083091510864
:1077600030931C0820931B0837FF08C088279927EF
:10777000821B930B90931C0880931B08209169082F
:1077800030916A08309346082093450837FF08C0B7
:1077900088279927821B930B90934608809345086E
:1077A0002091C40730E040E050E060912A047091DD
:1077B0002B0480912C0490912D040E94C457309387
:1077C000AF072093AE0737FF08C088279927821B91
:1077D000930B9093AF078093AE072091C40730E0DE
:1077E00040E050E0609132047091330480913404A1
:1077F000909135040E94C457A90137FF03C05095EA
:1078000041955F4F50931808409317088091AE0739
:107810009091AF07883C91050CF0EAC120911B08BC
:1078200030911C08283C31050CF0E2C160914508FC
:1078300070914608683C71050CF0DAC1483C51056E
:107840000CF0D6C1C901AA2797FDA095BA2F48EC24
:10785000E42EF12C012D112DA8019701281B390BC5
:107860004A0B5B0BCB01AA2797FDA095BA2FE81A0C
:10787000F90A0A0B1B0BCA01B9010E945057A80153
:1078800097010E9450570E94505720E034E244EF85
:1078900050E00E94C45720935308309354084093FB
:1078A00055085093560820916604309167048091E2
:1078B000DF039091E003281B390B37FF03C030959D
:1078C00021953F4F263031050CF09CC180918204F8
:1078D000909183044396879708F0A0C08091730429
:1078E000909174048F3F91052CF401969093740449
:1078F00080937304809173049091740402970CF444
:10790000A1C0609128087091290880912A0890915F
:107910002B082BE035E040E050E00E94C457309344
:107920001C0820931B082091660430916704809105
:10793000AA079091AB07281B390B30934608209378
:1079400045085FEF2C34350734F428593E4F309307
:107950004608209345088091450890914608853B4C
:10796000910534F0885691409093460880934508DD
:1079700080911B0890911C08209145083091460881
:10798000821B930B2091530830915408DC01A29F75
:10799000C001A39F900DB29F900D112464E670E08A
:1079A0000E948F5770934608609345086B307105AD
:1079B00034F08AE090E090934608809345088091E7
:1079C000450890914608865F9F4F34F486EF9FEFFD
:1079D00090934608809345082091450830914608C9
:1079E0002115310579F1109228081092290810927A
:1079F0002A0810922B088091660490916704909356
:107A0000AB078093AA078091180490911904821BF8
:107A1000930B909319048093180414C0809166040A
:107A2000909167049093AB078093AA071092740417
:107A300010927304109228081092290810922A08B4
:107A400010922B0881E080937104009166041091DC
:107A5000670460916F08709170088091710890912F
:107A600072082BE035E040E050E00E94C457021B52
:107A7000130BC80168E671E00E948F5790931C08B1
:107A800080931B088B30910534F08AE090E090934E
:107A90001C0880931B0880911B0890911C08865F2E
:107AA0009F4F34F486EF9FEF90931C0880931B0840
:107AB00020911B0830911C08C9010197833B910557
:107AC00020F0FFEF2C343F07ECF4B901882777FD55
:107AD0008095982F97FF07C0909580957095619538
:107AE0007F4F8F4F9F4F2091530830915408409102
:107AF0005508509156080E94505724E630E040E067
:107B000050E025C0243B310534F4C9018C549F4F0B
:107B1000843B9105D0F5B901882777FD8095982F92
:107B200097FF07C090958095709561957F4F8F4F17
:107B30009F4F20915308309154084091550850911F
:107B400056080E9450572CE93FEF4FEF5FEF0E941D
:107B5000C457CA01B9012BE035E040E050E00E9473
:107B6000505720916F0830917008409171085091E2
:107B70007208260F371F481F591F20936F08309334
:107B80007008409371085093720880916F0890912B
:107B90007008A0917108B0917208B7FF0CC08858A6
:107BA000984EA84FBF4F80936F0890937008A09392
:107BB0007108B093720880916F0890917008A0913D
:107BC0007108B0917208893727E1920727E0A20770
:107BD00020E0B207BCF088579741A740B04080939F
:107BE0006F0890937008A0937108B09372080AC050
:107BF00010927104109228081092290810922A08F5
:107C000010922B0880916604909167049093E00392
:107C10008093DF03E091B007F0E0EE0FFF1FE25822
:107C2000F84F2081318180916C0890E037FF03C0CC
:107C3000309521953F4F281739070CF046C0E09149
:107C4000B107F0E0EE0FFF1FE258F84F0190F0810E
:107C5000E02DF7FF03C0F095E195FF4FE817F90716
:107C6000A4F58091DD089091DE08892B71F12091B7
:107C700013082B3A80F08091B80785FF0CC08091E3
:107C8000E1039091E203892B31F0809172048330FB
:107C900091F084E014C02A3AC0F48091B80785FFBF
:107CA00014C08091E1039091E203892B71F08091DF
:107CB0007204843019F41092720403C083E080933C
:107CC00072048091720490E008C08091720488234D
:107CD00031F01092720480E090E00E94024A80919C
:107CE000C8089091C908892B29F08091C7048C306D
:107CF00009F44298809182049091830497FF03C015
:107D0000909581959F4F40976CF088EE93E090930B
:107D10009403809393038091B80784FD03C081E0AE
:107D20008093C604F090C107C0908204D090830471
:107D3000B601882777FD8095982F2F2D30E040E001
:107D400050E00E945057F601D7FE04C0EE27FF27EF
:107D5000EC19FD099F01442737FD4095542F0E94DF
:107D6000505720E032E040E050E00E94C4578901C3
:107D70009A018F2D90E0AC014C9DC0014D9D900D5E
:107D80005C9D900D112464E070E00E948F57600F9D
:107D9000711F882777FD8095982F6093DF0470937B
:107DA000E0048093E1049093E20420915A0430911E
:107DB0005B0440915C0450915D04261B370B480B1B
:107DC000590B20935A0430935B0440935C04509306
:107DD0005D042155334C4040504064F080E593EC05
:107DE000A0E0B0E080935A0490935B04A0935C04FD
:107DF000B0935D0480915A0490915B04A0915C045F
:107E0000B0915D04805B9C43AF4FBF4F64F480EB47
:107E10009CE3AFEFBFEF80935A0490935B04A09371
:107E20005C04B0935D048091C604882351F0809176
:107E3000660490916704909369048093680410929B
:107E4000C6048091A503282F30E030931C082093AE
:107E50001B082115310581F180917104882361F19E
:107E60008091B80783FF28C080916A0490916B04C9
:107E7000AC01249FC001259F900D349F900D1124CB
:107E800060E270E00E948F57882777FD8095982FD9
:107E900020915A0430915B0440915C0450915D0440
:107EA000260F371F481F591F20935A0430935B0435
:107EB00040935C0450935D048091C704815080938B
:107EC000C7048F5F09F0E8C088E18093C704809100
:107ED000D9039091DA0320910B0330910C03822394
:107EE0009323892B29F488B194E0892788B907C0A6
:107EF00080918604882311F0429A01C04298E09054
:107F0000C407FF2400E010E060912A0470912B0464
:107F100080912C0490912D04A80197010E94C457D0
:107F20003093230720932207609132047091330429
:107F30008091340490913504A80197010E94C457A0
:107F40003093250720932407809150089091510881
:107F500090932707809326078091690890916A087B
:107F6000909329078093280780915B0890915C0883
:107F700090932B0780932A0780918704909188041F
:107F800090932D0780932C0780916604909167044D
:107F9000909339078093380760916F08709170084B
:107FA00080917108909172082BE035E040E050E03C
:107FB0000E94C457309333072093320780911103F6
:107FC00090911203909335078093340780917D043C
:107FD00080933607109237078091430890914408A8
:107FE00090935107809350078091480890914908D9
:107FF000909353078093520780911D0890911E081B
:1080000090935507809354078091E6089091E70874
:1080100090935707809356078091E8089091E9085C
:1080200090935907809358078091EA089091EB0844
:1080300090935B0780935A078091EF089091F00826
:108040009C0103E0220F331F0A95E1F7880F991F67
:10805000280F391F8091C8089091C908280F391F2F
:108060008091720442E3849FC0011124280F391FBC
:1080700030935D0720935C078091F3049091F404A2
:1080800090935F0780935E078091F5049091F604CA
:10809000909361078093600780918F048823A9F0F3
:1080A0006091150870911608882777FD8095982FA4
:1080B0000E94395620916008309161084091620811
:1080C000509163080E94ED5632C0E0901508F09080
:1080D000160860912A0470912B0480912C049091D1
:1080E0002D040E94395620913B0830913C08409164
:1080F0003D0850913E080E94ED565B016C0100273F
:10810000F7FC0095102FC801B7010E943956209145
:1081100060083091610840916208509163080E94A4
:10812000ED569B01AC01C601B5010E9436550E9477
:108130000656709316086093150880919004882362
:10814000A9F06091090870910A08882777FD809549
:10815000982F0E9439562091600830916108409113
:108160006208509163080E94ED5632C0E090090801
:10817000F0900A08609132047091330480913404C5
:10818000909135040E94395620913B0830913C086B
:1081900040913D0850913E080E94ED565B016C01F4
:1081A0000027F7FC0095102FC801B7010E9439562F
:1081B00020916008309161084091620850916308F5
:1081C0000E94ED569B01AC01C601B5010E943655D7
:1081D0000E94065670930A086093090860915B0834
:1081E00070915C08882777FD8095982F0E943956FA
:1081F0007B018C0160916008709161088091620838
:10820000909163089B01AC010E9436559B01AC0123
:10821000C801B7010E94ED567B018C0160914604B4
:108220007091470480914804909149040E94395606
:1082300020913B0830913C0840913D0850913E0808
:108240000E94ED5620E030E040E05FE30E94ED56F2
:108250009B01AC01C801B7010E9436550E94065629
:1082600070935C0860935B088091150890911608E4
:1082700090934D0780934C078091090890910A08CC
:1082800090934F0780934E078091150890911608A0
:108290008150904434F080E090E4909316088093ED
:1082A000150880911508909116088050904C34F470
:1082B00080E090EC9093160880931508809109084F
:1082C00090910A088150904434F080E090E49093BB
:1082D0000A08809309088091090890910A08805043
:1082E000904C34F480E090EC90930A088093090855
:1082F00080915B0890915C088150904434F080E05C
:1083000090E490935C0880935B0880915B08909167
:108310005C088050904C34F480E090EC90935C08C2
:1083200080935B08C980DA80CC0CDD1CCC0CDD1C92
:108330008091B80780FF12C181FF4BC08091F50783
:108340009091A20384FF04C091559B3318F03AC06A
:108350009233C0F58091AF0381508093AF038F5F5C
:1083600009F052C08091170390911803895E9340E1
:1083700020F09091F8039A500AC0809117039091D1
:1083800018038436910588F49091F803965F9093D2
:10839000F80380917107891B87BD8CE291E090936F
:1083A000DA038093D9038AEF11C0809187049091FA
:1083B0008804449790938A048093890410926D04F2
:1083C00081E004C081E080936D0488EC8093AF036A
:1083D0001BC08091A2032091AD033091AE03280F02
:1083E000311D8091BD0790E0AC01249FC001259F05
:1083F000900D349F900D1124449790938A0480939C
:10840000890481E080936D0480916C04882321F0BD
:1084100010928A0410928904209187043091880474
:108420004091890450918A04421753070CF096C07A
:1084300080916D04882309F491C08091A30390E09A
:10844000241B350BDC01A29FC001A39F900DB29F9E
:10845000900D112464E070E00E948F574B01A090B2
:10846000F903B090FA036091620470916304809103
:10847000640490916504E090A403FF2400E010E000
:1084800020E830E040E050E00E94C457C801B70146
:108490000E94505720E230E040E050E00E94C45774
:1084A000F901BEEF283E3B0714F4E8EEFEEF8091A1
:1084B000C8049091C9049C01A4E0220F331FAA951F
:1084C000E1F7281B390BC50162E070E00E948F576D
:1084D000261B370B28193909CF01E1E089319E07A6
:1084E00014F088E191E0281B390BC9018C0D9D1D0A
:1084F00060E170E00E948F577093C9046093C804D4
:108500002091B90730E0220F331F220F331F62176B
:108510007307ACF4C216D30624F03093C904209339
:10852000C8048091B90790E0880F991F880F991FA0
:10853000C816D90624F4D092C904C092C804809108
:10854000C8049091C904C816D90624F4D092C9046D
:10855000C092C804C090C804D090C90480915A0841
:1085600090E04497880F991F880F991F46018C153A
:108570009D050CF44C0190923107809230070091D8
:108580005B0810915C086091DF047091E0048091B9
:10859000E1049091E2042CEF3FEF4FEF5FEF0E9478
:1085A0005057060F171FF1EA8F169104A4F094019B
:1085B00035952795021713070CF49801C40162E062
:1085C00070E00E948F57709561957F4F261737078F
:1085D0007CF49B010DC0C8012FEF003B120714F47F
:1085E00080EB9FEF9C018135910514F020E530E090
:1085F00080915A0890E0880F991F880F991FAC014D
:1086000048195909421753070CF49A01A401481B51
:10861000590B3901241735070CF43A0180911508DC
:108620009091160840907E0450907F04841995091B
:1086300090932D0880932C08E0903B08F0903C0824
:1086400000913D0810913E0820E030E040E050E00D
:10865000C801B7010E949A558823D1F16091E704BF
:108660007091E8048091E9049091EA040E943956DF
:108670005B016C0160912A0470912B0480912C04A1
:1086800090912D040E943956A80197010E94ED5641
:108690007B018C01B201882777FD8095982F0E947D
:1086A00039569B01AC01C801B7010E9435559B01A9
:1086B000AC01C601B5010E9436550E940656609372
:1086C000E7047093E8048093E9049093EA041CC0E3
:1086D00020912C0830912D08442737FD4095542FC8
:1086E0008091E7049091E804A091E904B091EA0434
:1086F000820F931FA41FB51F8093E7049093E80493
:10870000A093E904B093EA048091E7049091E8040F
:10871000A091E904B091EA0481509A4FA040B04082
:1087200064F080E09AEFA0E0B0E08093E7049093DB
:10873000E804A093E904B093EA048091E7049091DF
:10874000E804A091E904B091EA0480509640AF4F4C
:10875000BF4F64F480E096E0AFEFBFEF8093E70493
:108760009093E804A093E904B093EA0460912C0884
:1087700070912D08882777FD8095982F0E94395693
:108780007B018C016091E7047091E8048091E90419
:108790009091EA040E94395620919D0330919E03E6
:1087A00040919F035091A0030E94ED569B01AC01A4
:1087B000C801B7010E9436550E9406568B01C301BD
:1087C00077FE04C08827992786199709959587957C
:1087D000880D991D1C01442437FC4094542C209191
:1087E000AC0330E040E050E0C201B1010E945057BC
:1087F00020E430E040E050E00E94C457A901622F1D
:10880000232F041715071CF4C801602F292FEE270A
:10881000FF27E41BF50B862F922F8C010E171F07E5
:108820000CF48F01F301E80DF91DCF01800F911FAA
:1088300064E070E00E948F5777FF03C060E070E053
:1088400007C080915A0890E0861797070CF4BC0186
:1088500080911A0890E0681779070CF4BC016093C6
:108860000B08CF01801B910B64E070E00E948F57D2
:1088700077FF03C060E070E007C080915A0890E085
:10888000861797070CF4BC0180911A0890E06817CE
:1088900079070CF4BC016093140880910908909149
:1088A0000A0820918004309181043A8B298B821B25
:1088B000930B9093080880930708E0903B08F09092
:1088C0003C0800913D0810913E0820E030E040E077
:1088D00050E0C801B7010E949A558823E1F16091E8
:1088E000E3047091E4048091E5049091E6040E9411
:1088F00039565B016C0160913204709133048091B0
:108900003404909135040E943956A80197010E94C1
:10891000ED567B018C0149895A89BA01882777FD78
:108920008095982F0E9439569B01AC01C801B70170
:108930000E9435559B01AC01C601B5010E94365518
:108940000E9406566093E3047093E4048093E50468
:108950009093E6041CC02091070830910808442732
:1089600037FD4095542F8091E3049091E404A09149
:10897000E504B091E604820F931FA41FB51F8093F6
:10898000E3049093E404A093E504B093E60480919B
:10899000E3049091E404A091E504B091E6048150D1
:1089A0009A4FA040B04064F080E09AEFA0E0B0E0C1
:1089B0008093E3049093E404A093E504B093E60469
:1089C0008091E3049091E404A091E504B091E60461
:1089D00080509640AF4FBF4F64F480E096E0AFEF19
:1089E000BFEF8093E3049093E404A093E504B09375
:1089F000E6046091070870910808882777FD809544
:108A0000982F0E9439567B018C016091E30470918C
:108A1000E4048091E5049091E6040E943956209187
:108A20009D0330919E0340919F035091A0030E94AB
:108A3000ED569B01AC01C801B7010E9436550E945A
:108A400006567B018C012091AC0330E040E050E001
:108A5000C201B1010E94505720E430E040E050E0F4
:108A60000E94C457C901422F232FE816F90614F4B7
:108A70004E2D2F2D66277727681B790B842F922F79
:108A8000FC01E617F7070CF4FB01C40186199709EE
:108A90008E0F9F1F64E070E00E948F5777FF03C026
:108AA00060E070E007C080915A0890E08617970751
:108AB0000CF4BC0180911A0890E0681779070CF457
:108AC000BC0160934C088E1A9F0AC401861997094D
:108AD00064E070E00E948F5777FF03C060E070E0B1
:108AE00007C080915A0890E0861797070CF4BC01E4
:108AF00080911A0890E0681779070CF4BC01609324
:108B00003F0862960FB6F894DEBF0FBECDBFCF917F
:108B1000DF911F910F91FF90EF90DF90CF90BF906A
:108B2000AF909F908F907F906F905F904F903F900D
:108B30002F90089588EE8093B8073EE13093B907EF
:108B40008BEF8093BB078AE08093BC073093BA0712
:108B50003093BE0783E08093BD0758E05093BF0772
:108B600090E19093C00766E06093C1075093C207FD
:108B700086EE8093C3073093C40780E88093C507CF
:108B800044E64093C60788E78093C7078EE5809345
:108B9000C80783E28093C90784E18093CA071092D3
:108BA000CB079093CC071092CD071092CE0710926E
:108BB000CF071092D0071092E0071092E1071092B1
:108BC000E2071092E3074093D10788E28093D2072F
:108BD0001092F60792E39093D30786E98093D40727
:108BE00085E08093D5079093D6072AE52093D70791
:108BF0009093D8071092F5072093D9078093DA074E
:108C000085E58093DB078093DC0780E28093DD07B6
:108C100084E08093DE079093DF078FE58093E4077D
:108C200083EF8093E6073093E5073093E7078DEFF6
:108C30008093E8074093E9072093EA072093EB0726
:108C40002093EC071092ED076093EE075093EF0727
:108C50002093F0073093F1074093F2078CE3809361
:108C6000F307ABEFB7E0E8E7F3E08CE001900D929B
:108C70008150E1F7089588E68093B8074EE140936C
:108C8000B9078BEF8093BB078AE08093BC074093C2
:108C9000BA074093BE0783E08093BD078CE08093C2
:108CA000BF0780E18093C00776E07093C10768E05A
:108CB0006093C20786EE8093C3074093C40780E8A1
:108CC0008093C50780E58093C60788E78093C70730
:108CD0008EE58093C80783E28093C9074093CA0753
:108CE0001092CB0750E25093CC071092CD07109210
:108CF000CE071092CF071092D0071092E007109283
:108D0000E1071092E2071092E30734E63093D107AF
:108D100088E28093D2071092F60792E39093D307EC
:108D200086E98093D40785E08093D5079093D60792
:108D30002AE52093D7079093D8071092F507209340
:108D4000D9078093DA0785E58093DB078093DC07FA
:108D50005093DD0784E08093DE078BE48093DF0788
:108D60008FE58093E40783EF8093E60784E18093A7
:108D7000E5078093E7078DEF8093E8073093E907D5
:108D80002093EA072093EB072093EC071092ED075E
:108D90007093EE076093EF072093F0074093F1077D
:108DA0003093F2078CE38093F307ABEFB7E0E2E890
:108DB000F3E08CE001900D928150E1F7089588E690
:108DC0008093B8073EE13093B9078BEF8093BB07E0
:108DD0008AE08093BC073093BA073093BE0764E003
:108DE0006093BD075FE05093BF073093C0078CE0EE
:108DF0008093C10778E07093C20786EE8093C30723
:108E00003093C40780E88093C50780E58093C60748
:108E100096E99093C7078EE58093C80783E2809315
:108E2000C9073093CA071092CB0780E28093CC0722
:108E30001092CD071092CE071092CF071092D00754
:108E40001092E0071092E1071092E2071092E307F8
:108E500044E64093D10788E28093D2071092F60748
:108E600082E38093D3079093D40725E02093D5071E
:108E70008093D6079AE59093D7078093D8071092EE
:108E8000F5079093D9072093DA0785E58093DB07F0
:108E90008093DC0780E18093DD076093DE074093D9
:108EA000DF078FE58093E40783EF8093E607509315
:108EB000E5075093E7078DEF8093E8074093E907B4
:108EC0009093EA079093EB079093EC071092ED07CD
:108ED00086E08093EE077093EF079093F00730934E
:108EE000F1074093F2078CE38093F307ABEFB7E011
:108EF000EAE8F3E08CE001900D928150E1F70895EB
:108F00001092FC041092FB041092C9081092C80839
:108F10001092F0081092EF081092B40810929A087C
:108F2000109201091092C7081092DC081092EC0808
:108F30001092F4041092F3041092F6041092F504C7
:108F40001092EE081092ED081092DE081092DD08E3
:108F500008958091B408882309F4A6C080916B0815
:108F600065E00E946F57809331051092320588E0CA
:108F700090E0A0E0B0E080932D0590932E05A093A3
:108F80002F05B093300580910109882309F48CC026
:108F900080919A08882309F487C08091F50890E0B1
:108FA0008370907002970CF474C08091F60880FF73
:108FB00070C0109201096091A6087091A708809175
:108FC000A8089091A9082AE030E040E050E00E9413
:108FD000C4572093CA083093CB084093CC085093D1
:108FE000CD086091AA087091AB088091AC0890916F
:108FF000AD082AE030E040E050E00E94C4572093E2
:10900000CE083093CF084093D0085093D108609198
:10901000AE087091AF088091B0089091B1082AE035
:1090200030E040E050E00E94C4572093D2083093D3
:10903000D3084093D4085093D5081092B408809177
:109040008A0890918B08A0918C08B0918D0880932C
:10905000D6089093D708A093D808B093D908609108
:109060008E0870918F08809190089091910820EA65
:1090700036E841E050E00E94C4573093DB0820936B
:10908000DA0810929A0881E08093DC0820E030E052
:109090000DC01092DC0810929A08109201091092EB
:1090A000B40822E030E002C021E030E0C9010895B8
:1090B0000E94A9479C01181619060CF44CC0809117
:1090C000DD089091DE0823E0883E920730F4885A4C
:1090D0009D4F9093DE088093DD088091C708882318
:1090E000B1F18091CA089091CB082091B5083091D8
:1090F000B608821B930B9093E7088093E608809153
:10910000CE089091CF082091B9083091BA08821BFF
:10911000930B9093E9088093E8088091D20890918E
:10912000D3082091BD083091BE08821B930B909309
:10913000EB088093EA0881E08093EC0881E090E0FE
:109140009093EE088093ED0820E030E004C0109288
:10915000EC0822E030E0C90108950E94A947892B5C
:1091600099F58091CA089091CB08A091CC08B09154
:10917000CD088093B5089093B608A093B708B09334
:10918000B8088091CE089091CF08A091D008B091F6
:10919000D1088093B9089093BA08A093BB08B09304
:1091A000BC088091D2089091D308A091D408B091C6
:1091B000D5088093BD089093BE08A093BF08B093D4
:1091C000C00881E08093C7080895482F2091FB04D0
:1091D0003091FC042530310509F49DC0263031055D
:1091E0008CF42130310529F1223031051CF4232B78
:1091F000D1F003C12230310571F12330310509F07E
:10920000FCC02FC02730310509F4E2C027303105FA
:109210000CF492C02830310509F4E5C0293031053D
:1092200009F0EBC0A2C0853B09F0E7C081E090E007
:10923000D5C0823639F482E090E09093FC048093AC
:10924000FB0404C01092FC041092FB0410920D0564
:1092500010920E050895813009F0CFC083E090E0B0
:10926000BDC0883031F0823169F1833009F047C0E8
:1092700013C024EB38E03093280520932705809114
:10928000B4088823E1F5225130403093260520931D
:1092900025052E5E3F4F28C081E099E09093280578
:1092A0008093270580910109882349F581EF98E093
:1092B0009093260580932505409690931A058093F8
:1092C000190516C02AE938E03093280520932705B0
:1092D00080919A08882399F42452304030932605CF
:1092E000209325052C5D3F4F30931A0520931905D7
:1092F00085E090E09093FC048093FB0404C01092FE
:10930000FC041092FB04842F8F5F80930D058F5F08
:1093100080930E050895809317051092180580918B
:109320000D05840F80930D0590910E05980F909375
:109330000E0586E090E052C0382F20E0809117059E
:1093400090911805820F931F90931805809317052D
:1093500090910D05940F90930D0580910E05890F46
:1093600080930E0589E090E039C0609117057091F7
:1093700018056115710509F440C0E0912505F091CB
:109380002605808380910D05840F80930D059091B3
:109390000E05980F90930E05CB0101979093180539
:1093A00080931705892B89F08091190590911A05F2
:1093B0008E179F0750F03196F0932605E093250510
:1093C0003093FC042093FB04089587E090E006C0EE
:1093D00080910D05481789F488E090E09093FC0493
:1093E0008093FB04089580910E05481731F4E091B5
:1093F0002705F091280581E080831092FC041092EB
:10940000FB0408952F923F924F925F926F927F924A
:109410008F929F92AF92BF92CF92DF92EF92FF9284
:109420000F931F93DF93CF93CDB7DEB7E8970FB6B7
:10943000F894DEBF0FBECDBF9EAB8DAB83309105E0
:1094400009F4B2C08430910521F0892B09F414C1CC
:109450003CC78091C8089091C9080197029708F409
:1094600020C180910B0590910C05019690930C05FD
:1094700080930B058536910508F42AC710920C05D8
:1094800010920B051092200510921F0510922205D4
:1094900010922105109224051092230510920005C8
:1094A0001092FF041092FE041092FD0410920F051A
:1094B00010921005109211051092120510921305CA
:1094C00010921405109215051092160510920305BE
:1094D00010920405109205051092060510920705DA
:1094E000109208051092090510920A0510922A059B
:1094F0001092290510920205109201051092F008B1
:109500001092EF088091EC08882309F44AC08091FA
:10951000E6089091E7089093E0088093DF08609157
:10952000E8087091E9087093E2086093E10821E08F
:109530002093E50890939C0880939B0870939E0865
:1095400060939D082093A108709561957F4F909539
:1095500081959F4F0E94721B9C018091DF08909122
:10956000E00897FF03C08AE590E002C08EE091E03A
:10957000821B930B90931C0580931B0540911B0548
:1095800050911C056091E1087091E2088091DF081C
:109590009091E0080E94B21C70931E0560931D0517
:1095A00089C61092E5088DC68091C8089091C908B7
:1095B000019709F476C080910B0590910C050196F6
:1095C00090930C0580930B058955924008F480C652
:1095D00010920C0510920B058091EC08882309F479
:1095E00048C0109222051092210510922405109275
:1095F0002305109200051092FF041092FE041092B1
:10960000FD0410920F051092100510921105109292
:109610001205109213051092140510921505109260
:10962000160510920305109204051092050510927C
:109630000605109207051092080510920905109270
:109640000A0510922C0510922B058091E608909146
:10965000E70890939C0880939B088091E80890917C
:10966000E90890939E0880939D0881E08093A1086B
:1096700091C11092A10825C610920C0510920B05FD
:109680001092F4041092F3041092F6041092F50470
:109690001092F0081092EF081092C9081092C808B2
:1096A0001AC68091C8089091C9088130910509F4C3
:1096B00074C18230910541F0892B09F002C61092E5
:1096C0000C0510920B0507C68091E508882309F464
:1096D000F8C58091ED089091EE08181619060CF067
:1096E00059C18091EF089091F008099709F452C18F
:1096F00080911F05909120050196909320058093FD
:109700001F0560919B0870919C088091E6089091DC
:10971000E708AB01481B590B57FF03C05095419513
:109720005F4F20919D0830919E088091E8089091AC
:10973000E908281B390B37FF03C0309521953F4FAF
:10974000E0912905F0912A0580911D0590911E0553
:109750008E1B9F0B813591050CF44CC0443651058E
:1097600064F4243631054CF4809101059091020592
:109770008E309105CCF4029613C0483C51050CF58F
:10978000283C3105F4F48091010590910205883060
:10979000910514F0019704C08730910529F00196D6
:1097A0009093020580930105809101059091020537
:1097B0008E0F9F1F90932A058093290583E090E0E8
:1097C0000EC08091010590910205823091052CF028
:1097D0000197909302058093010584E090E09093B7
:1097E000F0088093EF0881E090E090932405809347
:1097F000230522C0C3970CF476C0443651055CF4AF
:109800002436310544F43A96F0932A05E09329056D
:1098100085E090E007C03196F0932A05E093290592
:1098200086E090E09093F0088093EF081092240572
:109830001092230581E090E090932205809321050A
:10984000A0902905B0902A05CC24B7FCC094DC2C4C
:1098500080911B0590911C050E94501C7C0120905A
:10986000290530902A05442437FC4094542C8091DB
:109870001B0590911C050E94A91C3C010027F7FCC8
:109880000095102FC801B701A60195010E945057FD
:1098900028EE33E040E050E00E94C4578091DF089A
:1098A0009091E008820F931F90939C0880939B08EF
:1098B000882477FC8094982CC401B301A201910103
:1098C0000E94505728EE33E040E050E00E94C45719
:1098D0008091E1089091E208820F931F90939E0877
:1098E00080939D0857C0443651050CF04DC0243676
:1098F00031050CF049C087E090E09093F008809328
:10990000EF08109222051092210510922405109262
:109910002305633071051CF06350704006C01FEFD3
:109920006E3F710734F46D5F7F4F70939C086093B6
:109930009B0880919D0890919E088330910514F0BA
:10994000039705C02FEF8E3F92072CF40396909358
:109950009E0880939D0880919B0890919C08039697
:109960000797C0F480919D0890919E0803960797F1
:1099700088F410929C0810929B0810929E081092F6
:109980009D0889E090E002C088E090E09093F008A4
:109990008093EF0881E090E08FC48091ED08909172
:1099A000EE08181619060CF081C480912B059091D1
:1099B0002C05019690932C0580932B054091E60889
:1099C0005091E70880919B0890919C08481B590B87
:1099D0005CAB4BABCA01AA2797FDA095BA2F8FA706
:1099E00098ABA9ABBAABA091E808B091E908809117
:1099F0009D0890919E08A81BB90BBEA7ADA77D013D
:109A00000027F7FC0095102FE9A6FAA60BA71CA7C4
:109A1000E0903105F09032050027F7FC0095102FFB
:109A20006FA578A989A99AA9A80197010E94505702
:109A3000DC01CB016AE070E00E948F576B018091DE
:109A4000FF0490910005C80ED91ED0920005C09267
:109A5000FF0469A57AA58BA59CA5A80197010E9482
:109A60005057DC01CB016AE070E00E948F578B01F8
:109A70008091FD049091FE04080F191F1093FE04BD
:109A80000093FD0420917E0830917F08409180086A
:109A90005091810829873A874B875C8780917A08A3
:109AA00090917B08A0917C08B0917D088D839E8366
:109AB000AF83B8871092EE081092ED08F090190865
:109AC000FF2009F44DC060912D0570912E05809105
:109AD0002F059091300520E43BE040E050E00E94EB
:109AE00050572F2D30E040E050E00E94C457C6018F
:109AF000D7FE04C0882799278C199D092817390794
:109B000054F0C80117FF04C088279927801B910BC8
:109B100028173907F4F4C601880F991F8C0D9D1D75
:109B2000880F991F68E070E00E948F5770930005BE
:109B30006093FF04C801880F991F800F911F880F41
:109B4000991F68E070E00E948F577093FE04609345
:109B5000FD0480912305909124051816190644F4FC
:109B6000109200051092FF041092FE041092FD0462
:109B70002091FF0430910005309327082093260898
:109B8000A090FD04B090FE04B0924108A09240085D
:109B9000E0901908FF2400E010E0442737FD4095CD
:109BA000542FC801B7010E94505720E830E040E030
:109BB00050E00E94C45739014A01CC24B7FCC0943C
:109BC000DC2CC601B501A80197010E94505720E87E
:109BD00030E040E050E00E94C45779018A012090B3
:109BE0002D0530902E0540902F0550903005C20174
:109BF000B10128E130E040E050E00E9450575B01A5
:109C00006C0166157705880599052CF4698B7A8BAC
:109C10008B8B9C8B15C0C201B10128EE3FEF4FEF3B
:109C20005FEF0E945057698A7A8A8B8A9C8A6616EF
:109C300077068806990624F4698B7A8B8B8B9C8B2C
:109C4000AE14BF04C006D1062CF4AD86BE86CF8606
:109C5000D88A15C0C201B10128EE3FEF4FEF5FEF88
:109C60000E945057ED86FE860F87188BE616F70682
:109C70000807190724F46D877E878F87988BA0913A
:109C80002105B0912205B8AFAFAB8091310590911D
:109C90003205E09075081A161B060CF087C0E69492
:109CA000E694FF240027F7FC0095102F5C01CC24DC
:109CB000B7FCC094DC2CC601B50129853A854B85DB
:109CC0005C850E945057A80197010E94505720E9D7
:109CD00031E040E050E00E94C45739014A01C6011A
:109CE000B5012D813E814F8158850E945057A801B2
:109CF00097010E94505720E931E040E050E00E9477
:109D0000C45779018A01C201B10128E330E040E083
:109D100050E00E9450575B016C016615770588057D
:109D200099052CF4698F7A8F8B8F9C8F15C0C20197
:109D3000B10128EC3FEF4FEF5FEF0E945057698E63
:109D40007A8E8B8E9C8E661677068806990624F48A
:109D5000698F7A8F8B8F9C8FAE14BF04C006D1069B
:109D60002CF4AD8ABE8ACF8AD88E15C0C201B1014B
:109D700028EC3FEF4FEF5FEF0E945057ED8AFE8ACD
:109D80000F8B188FE616F7060807190724F46D8B5A
:109D90007E8B8F8B988F90910C0886E0989FC001E6
:109DA0001124959587959595879580C0E694E694BE
:109DB000FF240027F7FC0095102F5C01CC24B7FC92
:109DC000C094DC2CC601B50129853A854B855C859C
:109DD0000E945057A80197010E9450572AEF30E087
:109DE00040E050E00E94C45739014A01C601B50164
:109DF0002D813E814F8158850E945057A8019701BF
:109E00000E9450572AEF30E040E050E00E94C457D3
:109E100079018A016201510136E0AA0CBB1CCC1CFD
:109E2000DD1C3A95D1F7A614B704C804D9042CF464
:109E3000A98EBA8ECB8EDC8E15C0C201B10120EC8A
:109E40003FEF4FEF5FEF0E945057698E7A8E8B8EF7
:109E50009C8E661677068806990624F4698F7A8F99
:109E60008B8F9C8FAE14BF04C006D1062CF4AD8A34
:109E7000BE8ACF8AD88E15C0C201B10120EC3FEF57
:109E80004FEF5FEF0E945057ED8AFE8A0F8B188FBD
:109E9000E616F7060807190724F46D8B7E8B8F8B67
:109EA000988F80910C0890E0959587955C01CC2463
:109EB000B7FCC094DC2CE0903105F090320500270F
:109EC000F7FC0095102F6FA578A989A99AA9A80178
:109ED00097010E945057A60195010E94505720E912
:109EE00031E040E050E00E94C45739014A016092DD
:109EF000030570920405809205059092060569A5F8
:109F00007AA58BA59CA5A80197010E945057A60190
:109F100095010E94505720E931E040E050E00E9456
:109F2000C45779018A01E0920705F0920805009371
:109F3000090510930A05C201B10128E330E040E0B1
:109F400050E00E9450575B016C016615770588054B
:109F500099054CF4609303057093040580930505FF
:109F60009093060515C0C201B10128EC3FEF4FEFF9
:109F70005FEF0E945057661677068806990644F4EC
:109F8000609303057093040580930505909306057F
:109F9000AE14BF04C006D1064CF4A0920705B092DF
:109FA0000805C0920905D0920A0515C0C201B10189
:109FB00028EC3FEF4FEF5FEF0E945057E616F70691
:109FC0000807190744F46093070570930805809308
:109FD000090590930A058091030590910405A091CD
:109FE0000505B091060590931E0880931D082091E9
:109FF0000705309108054091090550910A053093F5
:10A000006E0820936D08E988FA880B891C89E80E90
:10A01000F91E0A1F1B1F898D9A8DAB8DBC8DE80E12
:10A02000F91E0A1F1B1FD801C701B095A095909576
:10A0300081959F4FAF4FBF4F80930F0590931005B1
:10A04000A0931105B0931205ED84FE840F85188945
:10A05000E20EF31E041F151F2D893E894F89588D6E
:10A06000E20EF31E041F151F57016801D094C0941F
:10A07000B094A094A11CB11CC11CD11CA0921305CA
:10A08000B0921405C0921505D0921605909344081D
:10A0900080934308B0924908A092480860916F08E5
:10A0A0007091700880917108909172082BE035E0F2
:10A0B00040E050E00E94C45779018A01C9010E9422
:10A0C000A91C98A38F8F80910F0590911005A091E6
:10A0D0001105B09112058DA39EA3AFA3B8A7C70128
:10A0E0000E94501C9E8F8D8F20912D0530912E0542
:10A0F00040912F055091300529833A834B835C832F
:10A1000060900F05709010058090110590901205D9
:10A11000C7010E94A91C8C01809113059091140520
:10A12000A0911505B091160589A39AA3ABA3BCA372
:10A13000C7010E94501C98AF8FAB20902D05309026
:10A140002E0540902F05509030058BA99CA997FFB4
:10A1500003C0909581959F4F8159914054F48DA5EE
:10A160009EA597FF03C0909581959F4F815991407F
:10A170004CF01092F6041092F5041092F404109230
:10A18000F3049FC0B801882777FD8095982FA4011C
:10A1900093010E9450577B018C01EFA9F8ADBF01DC
:10A1A000882777FD8095982F29A13AA14BA15CA122
:10A1B0000E945057E61AF70A080B190BC201B101A9
:10A1C00028EE33E040E050E00E9450579B01AC0184
:10A1D000C801B7010E94C457C901DA01803BFFEFF3
:10A1E0009F07FFEFAF07FFEFBF0724F480EB9FEF60
:10A1F000AFEFBFEF81359105A105B10524F080E5F2
:10A2000090E0A0E0B0E09093F6048093F504ED8C2C
:10A21000FE8CB701882777FD8095982F2DA13EA150
:10A220004FA158A50E9450577B018C012F8D38A15A
:10A23000B901882777FD8095982FA60195010E9486
:10A240005057E60EF71E081F191F69817A818B810E
:10A250009C8128E13CEF4FEF5FEF0E9450579B013C
:10A26000AC01C801B7010E94C457C901DA01803BA3
:10A270003FEF93073FEFA3073FEFB30724F480EBD3
:10A280009FEFAFEFBFEF81359105A105B10524F038
:10A2900080E590E0A0E0B0E09093F4048093F304B4
:10A2A0004DA95EA944305105B1F404C08DA99EA901
:10A2B000049789F482E090E09093C9088093C808DD
:10A2C0000AC01092C9081092C80822E030E005C008
:10A2D00021E030E002C020E030E0C901E8960FB68E
:10A2E000F894DEBF0FBECDBFCF91DF911F910F91CC
:10A2F000FF90EF90DF90CF90BF90AF909F908F90A6
:10A300007F906F905F904F903F902F90089584B111
:10A31000806A84B93D9A82E58CBD1DBC459A81E076
:10A32000809302098AEA8093060983E880930709EB
:10A330008AE08093080910920A0910920909109284
:10A340000C0910920B09109228091092290987E430
:10A3500080932A0987E080932B0983E080932C095E
:10A360000895F89460912A0470912B0480912C0434
:10A3700090912D042CE630E040E050E00E94C4575C
:10A3800030930A09209309096091320470913304D3
:10A3900080913404909135042CE630E040E050E0A8
:10A3A0000E94C45730930C0920930B0960916508F3
:10A3B0007091660880916708909168082BE035E0FD
:10A3C00040E050E00E94C4573093120920931109D5
:10A3D0002091220430912304809132089091330817
:10A3E000B9010E948F57CB01880F991F860F971FC5
:10A3F000880F991F880F991F90930E0980930D095C
:10A4000080915E0890915F08B9010E948F57CB013F
:10A41000880F991F860F971F880F991F880F991F04
:10A420009093100980930F09109223041092220434
:10A43000109233081092320810925F0810925E0852
:10A44000809108098C3009F4EAC08D3030F48A30EC
:10A4500051F08B3009F005C171C08D30F1F18E30B3
:10A4600009F0FFC0EEC08091950480931909809196
:10A47000960480931A098091970480931B09809118
:10A48000980480931C098091990480931D09809100
:10A490009A0480931E0980919B0480931F098091E8
:10A4A0009C04809320098091AB0480932109837FD1
:10A4B0008093AB0480911103909112038093220941
:10A4C0008091C80780932309F999FECF82E090E03C
:10A4D00092BD81BDF89A80B52EC08091E807809327
:10A4E00019098091E90780931A098091EA078093FE
:10A4F0001B098091EB0780931C098091EC078093E6
:10A500001D098091ED0780931E098091EE078093CD
:10A510001F098091EF07809320098091F2078093B3
:10A5200021098091F007809322098091F10780939F
:10A5300023098091F3078093240993C0E091B20727
:10A54000F0E0EE0FFF1FE258F84F0190F081E02D90
:10A550002FEFE138F20714F4E1E8FFEFE038F105FE
:10A5600014F0EFE7F0E0E0931909E091B307F0E0B1
:10A57000EE0FFF1FE258F84F0190F081E02D6FEFD2
:10A58000E138F60714F4E1E8FFEFE038F10514F0E4
:10A59000EFE7F0E0E0931A09E091B107F0E0EE0F89
:10A5A000FF1FE258F84F0190F081E02D8FEFE13866
:10A5B000F80714F4E1E8FFEFE038F10514F0EFE7F5
:10A5C000F0E0E0931B09E091B007F0E0EE0FFF1F11
:10A5D000E258F84F0190F081E02D2FEFE138F207BB
:10A5E00014F4E1E8FFEFE038F10514F0EFE7F0E0F4
:10A5F000E0931C098091750480931D098091770474
:10A6000080931E098091790480931F0980917B04B7
:10A610008093200980917D048093210922C080913C
:10A620007B06863018F010927B0685E0809319092E
:10A63000809187049091880490931C0980931B0952
:10A6400010C0809129098093190980912A0980936B
:10A650001A0980912B0980931B0980912C09809302
:10A660001C09789480912809882309F476C04091C8
:10A670002E0950912F09CA0181509E4F8F5F934040
:10A68000B0F42091300930913109C90181509E4FB9
:10A690008F5F934060F48091B80785FF08C05093A6
:10A6A000F4044093F3043093F6042093F50480916E
:10A6B00034099091350921E08936920724F490936A
:10A6C00067048093660480916604909167042091EA
:10A6D000680430916904845E9D4F821B930B68E689
:10A6E00071E00E948F57845B904090936B0480933D
:10A6F0006A0420913809309139098091D9039091E9
:10A70000DA038217930740F480917B06882321F4B3
:10A710003093DA032093D90380912D09843679F0A0
:10A720008736D9F480913A098093650980913B0975
:10A730008093670980913C09809366090895809110
:10A740003A09809361091092620980913C099091C5
:10A750003D099093640980936309089580910209EB
:10A76000882309F43BC0459886E099E0909304095A
:10A770008093030990913305E92FF0E0E055FC4FF9
:10A780008081809308099F5F90933305963010F085
:10A7900010923305109202090E94B15181E080931A
:10A7A000050900000000000000000000000000009B
:10A7B0000000000000000000000000000000000099
:10A7C0000000000000000000000000000000000089
:10A7D000000080910609809325098EBD089580911F
:10A7E0000209882309F07BC00DB407FE78C084E01D
:10A7F0008093DB03459A2EB580913505813069F051
:10A80000813018F08230C9F513C0109227092093C7
:10A810003405213891F581E008C0253541F5809156
:10A8200034058B5A8093340582E08093350525C02A
:10A8300080912709E82FF0E0E95BF64F20838F5FD6
:10A8400080932709909134058A31A0F0291769F483
:10A85000ADE2B9E0E7E4F9E08AE101900D928150C0
:10A86000E1F781E08093280902C010922809109234
:10A87000350503C0920F90933405209105092032CD
:10A8800008F027C04598000000000000000000000C
:10A8900000000000000000000000000000000000B8
:10A8A00000000000000000000000000000000000A8
:10A8B000000000000000E0910309F0910409E20F9C
:10A8C000F11D80818EBD90912509890F8093250906
:10A8D00003C081E0809302092F5F2093050908954A
:10A8E00087B18C6087B94298439810923A0580E806
:10A8F0008093B60310923B058093B703089580912F
:10A900003C05815080933C058F5F09F068C084E06E
:10A9100080933C058091E5078B3F80F0809134085F
:10A92000873E28F08091E40787FF25C022C08A3047
:10A9300028F48091E40787FF1CC01DC080913A0570
:10A94000815080933A058F5FB9F48091340881502B
:10A9500080933A058091B603813011F480E801C0FC
:10A9600086958093B6038091E4079091B60389237E
:10A9700011F0429A01C042988091E7078B3F88F01E
:10A9800080915908873E28F08091E60787FF07C02D
:10A9900023C08A3030F48091E60787FF1DC04398BA
:10A9A000089580913B05815080933B058F5FB9F4FA
:10A9B00080915908815080933B058091B703813085
:10A9C00011F480E801C086958093B7038091E60773
:10A9D0009091B703892311F0439A089543980895FD
:10A9E000FC014150504030F001900616D1F73197EC
:10A9F000CF010895882799270895A0E0B0E0E3E00B
:10AA0000F5E50C94E9577C01EB018A01690109C065
:10AA1000CE012196F6010995F70181937F0101503E
:10AA2000104001151105A1F7CDB7DEB7E8E00C9491
:10AA30000558A0E0B0E0EFE1F5E50C94E957EC0132
:10AA40007B018A01690109C0F70161917F01CE0193
:10AA50002196F60109950150104001151105A1F745
:10AA6000CDB7DEB7E8E00C9405585058BB27AA27AD
:10AA70000ED075C166D130F06BD120F031F49F3F1C
:10AA800011F41EF45BC10EF4E095E7FB51C1E92F10
:10AA900077D180F3BA17620773078407950718F018
:10AAA00071F49EF58FC10EF4E0950B2EBA2FA02DF8
:10AAB0000B01B90190010C01CA01A0011124FF276B
:10AAC000591B99F0593F50F4503E68F11A16F04066
:10AAD000A22F232F342F4427585FF3CF4695379565
:10AAE0002795A795F0405395C9F77EF41F16BA0B2A
:10AAF000620B730B840BBAF09150A1F0FF0FBB1FD8
:10AB0000661F771F881FC2F70EC0BA0F621F731F20
:10AB1000841F48F4879577956795B795F7959E3F7D
:10AB200008F0B3CF9395880F08F09927EE0F97950B
:10AB300087950895D9D008F481E008950CD00FC10D
:10AB400007D140F0FED030F021F45F3F19F0F0C0A3
:10AB5000511139C1F3C014D198F39923C9F3552386
:10AB6000B1F3951B550BBB27AA2762177307840700
:10AB700038F09F5F5F4F220F331F441FAA1FA9F3B6
:10AB800033D00E2E3AF0E0E830D091505040E695A8
:10AB9000001CCAF729D0FE2F27D0660F771F881F09
:10ABA000BB1F261737074807AB07B0E809F0BB0BF8
:10ABB000802DBF01FF2793585F4F2AF09E3F51051C
:10ABC00068F0B6C000C15F3FECF3983EDCF38695B9
:10ABD00077956795B795F7959F5FC9F7880F911D92
:10ABE0009695879597F90895E1E0660F771F881F7E
:10ABF000BB1F621773078407BA0720F0621B730B31
:10AC0000840BBA0BEE1F88F7E095089504D0689482
:10AC1000B111D9C00895BCD088F09F5790F0B92FDA
:10AC20009927B751A0F0D1F0660F771F881F991FA1
:10AC30001AF0BA95C9F712C0B13081F0C3D0B1E0B3
:10AC40000895C0C0672F782F8827B85F39F0B93FC3
:10AC5000CCF3869577956795B395D9F73EF49095A3
:10AC60008095709561957F4F8F4F9F4F0895E89421
:10AC700009C097FB3EF490958095709561957F4F44
:10AC80008F4F9F4F9923A9F0F92F96E9BB279395F2
:10AC9000F695879577956795B795F111F8CFFAF402
:10ACA000BB0F11F460FF1BC06F5F7F4F8F4F9F4F33
:10ACB00016C0882311F096E911C0772321F09EE891
:10ACC000872F762F05C0662371F096E8862F70E0F7
:10ACD00060E02AF09A95660F771F881FDAF7880FD1
:10ACE0009695879597F90895990F0008550FAA0B27
:10ACF000E0E8FEEF16161706E807F907C0F012168F
:10AD00001306E407F50798F0621B730B840B950B91
:10AD100039F40A2661F0232B242B252B21F40895E6
:10AD20000A2609F4A140A6958FEF811D811D089583
:10AD300097F99F6780E870E060E008959FEF80ECEE
:10AD4000089500240A941616170618060906089591
:10AD500000240A9412161306140605060895092EF7
:10AD60000394000C11F4882352F0BB0F40F4BF2B66
:10AD700011F460FF04C06F5F7F4F8F4F9F4F0895A6
:10AD800057FD9058440F551F59F05F3F71F047959C
:10AD9000880F97FB991F61F09F3F79F08795089581
:10ADA000121613061406551FF2CF4695F1DF08C0A0
:10ADB000161617061806991FF1CF869571056105BD
:10ADC00008940895E894BB2766277727CB0197F965
:10ADD00008958ADF08F48FEF08950BD0C0CFB1DF5C
:10ADE00028F0B6DF18F0952309F0A2CFA7CF1124E1
:10ADF000EACFC6DFA0F3959FD1F3950F50E0551F22
:10AE0000629FF001729FBB27F00DB11D639FAA27BF
:10AE1000F00DB11DAA1F649F6627B00DA11D661F0E
:10AE2000829F2227B00DA11D621F739FB00DA11D2F
:10AE3000621F839FA00D611D221F749F3327A00DE9
:10AE4000611D231F849F600D211D822F762F6A2F85
:10AE500011249F5750408AF0E1F088234AF0EE0F0A
:10AE6000FF1FBB1F661F771F881F91505040A9F717
:10AE70009E3F510570F05CCFA6CF5F3FECF3983E4C
:10AE8000DCF3869577956795B795F795E7959F5F7E
:10AE9000C1F7FE2B880F911D9695879597F9089518
:10AEA000629FD001739FF001829FE00DF11D649FAE
:10AEB000E00DF11D929FF00D839FF00D749FF00D3A
:10AEC000659FF00D9927729FB00DE11DF91F639FDB
:10AED000B00DE11DF91FBD01CF0111240895991B8B
:10AEE00079E004C0991F961708F0961B881F7A9581
:10AEF000C9F780950895AA1BBB1B51E107C0AA1F83
:10AF0000BB1FA617B70710F0A61BB70B881F991F0A
:10AF10005A95A9F780959095BC01CD01089597FBAE
:10AF2000092E07260AD077FD04D0E5DF06D00020E1
:10AF30001AF4709561957F4F0895F6F79095819575
:10AF40009F4F0895A1E21A2EAA1BBB1BFD010DC045
:10AF5000AA1FBB1FEE1FFF1FA217B307E407F507C9
:10AF600020F0A21BB30BE40BF50B661F771F881FA5
:10AF7000991F1A9469F760957095809590959B013B
:10AF8000AC01BD01CF01089597FB092E05260ED017
:10AF900057FD04D0D7DF0AD0001C38F450954095F7
:10AFA000309521953F4F4F4F5F4F0895F6F790959D
:10AFB0008095709561957F4F8F4F9F4F08952F9289
:10AFC0003F924F925F926F927F928F929F92AF9239
:10AFD000BF92CF92DF92EF92FF920F931F93CF9386
:10AFE000DF93CDB7DEB7CA1BDB0B0FB6F894DEBF1D
:10AFF0000FBECDBF09942A88398848885F846E8443
:10B000007D848C849B84AA84B984C884DF80EE808C
:10B01000FD800C811B81AA81B981CE0FD11D0FB695
:10B02000F894DEBF0FBECDBFED010895F894FFCFB9
:10B030000A010101FF6401C800496E74656772610D
:10B040006C4E69636B20202020496E7465677261C5
:10B050006C526F6C6C202020204163634E69636BDF
:10B06000202020202020202020416363526F6C6C20
:10B070002020202020202020204779726F476965FA
:10B08000722020202020202020486F6568656E57A0
:10B090006572742020202020204163635A202020E4
:10B0A00020202020202020202047617320202020E5
:10B0B00020202020202020202045727361747A4BAC
:10B0C0006F6D706173732020205370616E6E756EAA
:10B0D000672020202020202020456D7066616E674B
:10B0E0002020202020202020204B6F6D7061737362
:10B0F0002020202020202020204D6F746F725F566A
:10B100006F726E6520202020204D6F746F725F4833
:10B11000696E74656E202020204D6F746F725F4CD5
:10B12000696E6B7320202020204D6F746F725F5208
:10B130006563687473202020202020202020202098
:10B1400020202020202020202020202020202020FF
:10B1500020202020202020202020202020202020EF
:10B1600020202020202020202020202020202020DF
:10B1700020202020202020202020202020202020CF
:10B180002020202020202020204E69636B202020BA
:10B19000202020202020202020526F6C6C20202096
:10B1A00020202020202020202064656275675F30E9
:10B1B00020202020202020202064656275675F31D8
:10B1C00020202020202020202064656275675F32C7
:10B1D00020202020202020202075746D5F65617361
:10B1E00074202020202020202075746D5F6E6F72E7
:10B1F00074682020202020202075746D5F616C749D
:10B200002020202020202020204750535F537461AD
:10B210007465202020202020204750535F4E696312
:10B220006B20202020202020204750535F526F6C3D
:10B230006C20202020202020202800FFFF64008098
:10B24000016400007D0000FF0373737301020304B7
:10B2500005060708090A48616C6C6F2057656C7415
:10B2600000000000000000000000000000000000DE
:10B2700000000000000000000000000000000000CE
:10B2800000000000000000000000000000000000BE
:10B2900000000000000000000000000000000000AE
:10B2A0000000000000000B01426567696E6E657268
:10B2B00000004E6F726D616C000053706F7274000D
:10B2C000006400F40190D0030090D0030017B7D1C0
:10B2D0003830FB103A409696020A644664ECFF64EC
:08B2E0000A0B0D0B0C0E01011D
:00000001FF
